:100000000C9491010C94A3010C94A3010C94802EE8
:100010000C94722B0C94A3010C94A3010C94A301D7
:100020000C94A3010C94A3010C94A3010C948515CA
:100030000C94A3010C94A3010C94A3010C94A301B0
:100040000C9439150C94A3010C9485340C94DF3175
:100050000C94A3010C94A3010C94A3010C94A30190
:100060000C94A3010C94A3017903140F140F8303C0
:100070008E039903A403140FA803140FB603140FDF
:10008000C003CA03D403140F140F140FE403F103C5
:10009000FE031E14241427142A142F1437143F149B
:1000A000DA14DA14DA144C144F1458146114DA14F4
:1000B000DA14DA14DA14DA14DA146D1477148314F7
:1000C0008B148E149714A014A614DA14DA14AF1437
:1000D000B814C314BB34BD34F634F634F634F634F5
:1000E000F634F634F634F634F634F634C334C53424
:1000F000C734C934CB34CD34CF34D134F634D534CD
:10010000D734D934DB34DD34DF34F634E134084A13
:10011000D73B3BCE016E84BCBFFDC12F3D6C74311B
:100120009ABD56833DDA3D00C77F11BED9E4BB4C72
:100130003E916BAAAABE000000803F05A84CCDB23C
:10014000D44EB93836A9020C50B9918688083CA61D
:10015000AAAA2ABE000000803F00536C6565706942
:100160006E6700526573746F72696E672073706991
:100170006E646C6500526573746F72696E6720649B
:10018000656661756C74730050676D20456E640020
:10019000436865636B204C696D69747300436865DF
:1001A000636B20446F6F720044697361626C6564B5
:1001B00000456E61626C65640043617574696F6EC1
:1001C0003A20556E6C6F636B656400272448277C6A
:1001D0002724582720746F20756E6C6F636B005254
:1001E0006573657420746F20636F6E74696E7565D6
:1001F000005B4D53473A000D0A4772626C20312E66
:100200003166205B27242720666F722068656C703A
:100210005D0D0A00244E005B4F50543A005B56457A
:10022000523A312E31662E32303137303330323A55
:10023000005B544C4F3A005B4739323A0033300090
:100240003238005B4700204700204D00205300203B
:10025000460020540033382E005B47433A47005B8A
:10026000484C503A24242024232024472024492089
:10027000244E2024783D76616C20244E783D6C69B4
:100280006E6520244A3D6C696E652024534C5020D5
:100290002443202458202448207E2021203F20630E
:1002A00074726C2D785D0D0A00414C41524D3A003C
:1002B0007C413A007C4F763A007C57434F3A007CB1
:1002C000506E3A007C46533A007C42663A007C57B6
:1002D000506F733A007C4D506F733A00536C6565F4
:1002E0007000446F6F723A00436865636B00416C45
:1002F00061726D00486F6D65004A6F6700486F6CF2
:10030000643A0052756E0049646C65000D0A005B2A
:100310005052423A006572726F723A006F6B0D0A6A
:10032000000011241FBECFEFD8E0DEBFCDBF27E015
:10033000A0E0B1E001C01D92A136B207E1F70E9432
:10034000B90F0C94A53A0C9400002F923F924F9253
:100350005F926F927F928F929F92AF92BF92CF9255
:10036000DF92EF92FF920F931F93CF93DF93CDB75E
:10037000DEB7CA54D1090FB6F894DEBF0FBECDBFA9
:100380008AE3E0ECF1E0DF011D928A95E9F78BE06A
:10039000E0E8F1E0A1ECB1E001900D928A95E1F77F
:1003A00080911107843211F00C94350F81E0809315
:1003B000C1011092C20183E08A8FB1E0BBA3212C5E
:1003C000312C1CA61BA610E01B8E1F8EEE24E3947E
:1003D000F12CEAE0AE2EB12CF1E68F2EF3E09F2E49
:1003E0008A8DE82FF0E0EF5EF84FD080DD2009F431
:1003F00035C29FEB9D0D9A3110F00C94040F8F5F66
:100400008A8FBE016A5E7F4FCE014A960E942135D7
:10041000882311F40C94060F4E885F88688C798CC1
:10042000C301B2010E94103A0E944E37062F70E0BD
:1004300080E090E00E947F379B01AC01C301B201D4
:100440000E94D53520E030E048EC52E40E942D397E
:100450000E949A390E944E37CB01E7E4DE1629F05C
:10046000FDE4DF1609F4EAC033C1083209F4C6C05E
:1004700020F5043168F4013108F08AC0043009F431
:1004800052C008F464C00A3009F445C00C94140F3B
:100490000C3109F440C050F4063110F00C94140FE4
:1004A00025E1201B2093C30126E0ADC00E3199F158
:1004B000063209F44CC00C94140F0D3309F498C0A3
:1004C000A8F4053381F140F40B3209F47AC001330A
:1004D00009F477C00C94140F0C3310F00C94140F23
:1004E0006AEC600F6093C70129E08DC00C3538F4C9
:1004F0000A3508F053C0003581F10C94140F0C3507
:1005000051F00F3510F00C94140F2EE5201B2093A2
:10051000C20125E078C0009731F42F8D21110C9491
:10052000080F31E03F8F0093C001202F2D7F2C3129
:1005300019F00C3509F064C0009721F00A9711F00A
:100540000C94140F600F6093C00120E061C04F8DC8
:1005500041110C94080FA2E0AF8F0093C101063245
:1005600009F050C08431910559F08E31910541F068
:100570008832910529F08233910511F00C94140F03
:10058000B5010E94423A66576093C10121E040C024
:100590006FEE600F6093C50122E035C0892B31F406
:1005A00066EA600F6093C40123E032C06A307105CF
:1005B00011F00C94140F0A3511F40C94140F24E06C
:1005C00027C0BF8DB1110C94080F013331F4109284
:1005D000C60128E0E3E0EF8F1BC00A9711F00C94EE
:1005E000140FF1E0F093C60128E033E03F8F10C014
:1005F000892B11F00C94140F2AE00AC027E003C0E5
:1006000020E001C021E0892B19F087E10C943C0F18
:10061000C70102C0880F991F2A95E2F72BA53CA5B8
:1006200028233923232B19F085E10C943C0FABA52B
:10063000BCA5A82BB92BBCA7ABA7D2CE892B29F779
:10064000063018F4033058F016C0083010F40C943B
:10065000140F0A30F0F00E3159F00C94140F0023EF
:1006600019F0013001F104C0B3E0B093C8011BC020
:100670000093C80118C0043021F0053031F080E14A
:1006800001C080E28093CA0102C01092CA018CE0CE
:100690000BC0093021F080E48093C90102C01092A0
:1006A000C9018DE001C08BE0F70102C0EE0FFF1F12
:1006B0008A95E2F72BA53CA52E233F23232B09F097
:1006C000B3CF2BA53CA52E2B3F2B3CA72BA788CE29
:1006D0008D2DDD0C990BAA0BBB0BFC01E654F10927
:1006E000E531F10510F00C94140FEC5CFF4F0C9405
:1006F000783A4092CC015092CD016092CE01709236
:10070000CF0180E087C04092D0015092D101609229
:10071000D2017092D301116081E07CC04092D4017B
:100720005092D5016092D6017092D701126082E09A
:1007300071C04092D8015092D9016092DA01709252
:10074000DB01146083E066C00093DC0184E062C0DA
:10075000C301B2010E9447376093DD017093DE014F
:100760008093DF019093E00185E054C04092E10165
:100770005092E2016092E3017092E40186E04AC087
:100780004092E5015092E6016092E7017092E80123
:1007900087E040C04092E9015092EA016092EB018B
:1007A0007092EC0188E036C020E030E04FE753E47F
:1007B000C301B2010E94ED38181614F40C940A0F0C
:1007C0000093ED0189E026C04092EE015092EF01C6
:1007D0006092F0017092F1013B8D31603B8F8AE0B5
:1007E00019C04092F2015092F3016092F4017092AC
:1007F000F5014B8D42604B8F8BE00CC04092F601AF
:100800005092F7016092F8017092F9018B8D84602B
:100810008B8F8CE06701082E02C0CC0CDD1C0A9483
:10082000E2F7960122213321232B11F00C940C0FB7
:10083000D40102C0B595A7958A95E2F7A0FF0BC039
:1008400020E030E0A901C301B2010E94CB3687FF4E
:1008500002C00C940E0F2C283D28C2CDBB8DBB23AB
:1008600029F0EF8DE11102C0F2E0FF8F25FE0FC0ED
:100870008091DD019091DE01A091DF01B091E00156
:1008800081389649A849B10514F00C94100F3BA18A
:10089000332329F020FC02C00C941A0F18C0809159
:1008A000C201813071F44F8D4230E1F58091C10178
:1008B0008035C1F18823B1F120FC02C00C941A0FDD
:1008C00031C08091810181112DC020FE1BC080911B
:1008D000C301813039F523E333E34BEC51E46091FC
:1008E000CC017091CD018091CE019091CF010E94F9
:1008F0002D396093CC017093CD018093CE019093FC
:10090000CF0110C080918F0190919001A091910131
:10091000B09192018093CC019093CD01A093CE0130
:10092000B093CF0130FC10C080918B0190918C016D
:10093000A0918D01B0918E018093E9019093EA011D
:10094000A093EB01B093EC018091C001843039F4A5
:1009500026FC03C08CE10C943C0FE89426F88091AF
:10096000C501882369F0813029F48FAF1DAE92E074
:100970009BAF0BC01FAEA2E0ADAFB1E0BBAF05C0F7
:10098000E2E0EFAFF1E0FDAF1BAE8091C30181303B
:1009900021F02F8D2330C9F52FC060ECC62E61E009
:1009A000D62EE12CF12C3B8DA32EB12CC5010E2CA3
:1009B00002C0959587950A94E2F780FF12C023E361
:1009C00033E34BEC51E4D6019E966D917D918D9170
:1009D0009C91D1970E942D39F60166A777A780AB2D
:1009E00091ABFFEFEF1AFF0A24E0C20ED11C33E0F7
:1009F000E316F104D9F6CDCF8091C601813029F4F8
:100A00004B8D443011F00C94120F8CE0E4EAF1E0CD
:100A1000DE01119601900D928A95E1F78BA59CA5B8
:100A200091FD08C00091C0010A30C9F00C3509F4ED
:100A3000B3C01EC18091C701873018F08DE10C94BE
:100A40003C0F90918601891769F3BE016F5F7F4F5C
:100A50000E949D1E882311F40C94280FE3CF9B8DD8
:100A6000911103C08AE10C943C0FC1018075992754
:100A7000892B09F46FCF6091E1017091E2018091BF
:100A8000E3019091E4010E94103A0E944E376730D2
:100A9000A8F68091DC01843141F0823011F00C9491
:100AA000140F27FE02C00C94140FAFEA2A2266230B
:100AB00019F0615069A703C0B091C701B9A760EDF3
:100AC00071E089A50E949D1E882311F40C94280FC3
:100AD0000091DC014090BC015090BD016090BE01CE
:100AE0007090BF0140ECE42E41E0F42E50E8A52EBA
:100AF00051E0B52EC12CD12CEB8D8E2E912CC40142
:100B00000C2C02C0959587950A94E2F780FF35C0BA
:100B1000043151F5D501D0962D913D914D915C91C7
:100B2000D39758966D917D918D919C915B970E9482
:100B3000D535F70126A537A540A951A90E94D5357D
:100B4000D70150966D937D938D939C935397B2E00C
:100B5000CB1213C0A30192010E94D535F701608B1F
:100B6000718B828B938B09C0F70186A597A5A0A9ED
:100B7000B1A9808B918BA28BB38BFFEFCF1ADF0AC9
:100B800024E0E20EF11C34E0A30EB11C43E0C416D5
:100B9000D10409F0B4CF3FC18B8D882309F462CF13
:100BA0004090BC015090BD016090BE017090BF01AB
:100BB00020E8822E21E0922EDE0111967D0130EC9C
:100BC000C32E31E0D32EA12CB12CE82FF0E0F8A7F2
:100BD000EFA38FA198A50A2C02C0959587950A943A
:100BE000E2F780FF29C0D7012D913D914D915C9195
:100BF000F401608D718D828D938D0E94D535D60163
:100C00009E962D913D914D915C91D1970E94D53545
:100C1000F60166A777A780AB91ABF2E0AF1216C0E2
:100C2000A30192010E94D535D6019E966D937D93C6
:100C30008D939C93D1970AC0F40180A991A9A2A990
:100C4000B3A9F60186A797A7A0ABB1ABFFEFAF1A88
:100C5000BF0A24E0820E911C34E0E30EF11C44E054
:100C6000C40ED11C83E0A816B10409F0B2CFD2C0E3
:100C70009F8D933069F40E3109F494C0053309F463
:100C8000C3C00C3109F0C6C060ED71E086E08DC0D4
:100C9000AB8DAA2381F3B091C401BFA34090BC01E6
:100CA0005090BD016090BE017090BF0180E8A82EF9
:100CB00081E0B82E90ECE92E91E0F92EFE013196FC
:100CC0004F01C12CD12C2A2F30E03AA729A789A5A2
:100CD0009AA50C2C02C0959587950A94E2F780FDA1
:100CE0000BC0F501808D918DA28DB38DF70186A784
:100CF00097A7A0ABB1AB44C0053309F441C0FFA135
:100D0000F1112BC0D501D0962D913D914D915C9163
:100D1000D397F40160817181828193810E94D635DD
:100D2000D7019E962D913D914D915C91D1970E9456
:100D3000D635F70166A777A780AB91ABF2E0CF126B
:100D40001FC0A30192010E94D635D7019E966D93D4
:100D50007D938D939C93D19713C0F501208D318D98
:100D6000428D538DD7019E966D917D918D919C9171
:100D7000D1970E94D635F70166A777A780AB91ABD4
:100D8000FFEFCF1ADF0A24E0A20EB11C34E0E30E1D
:100D9000F11C44E0840E911C83E0C816D10409F0D4
:100DA00096CF69CF60ED71E087E00E949D1E882399
:100DB00011F40C94280F9B8D911103C019A61F8E5E
:100DC0002AC0A0E8B1E0E0ECF1E080E090E04B8DDB
:100DD000242F30E0A901082E02C0559547950A94AA
:100DE000E2F740FD0AC058964D915D916D917C915E
:100DF0005B97408B518B628B738B01961496349664
:100E00008330910539F706C08091C101823010F01E
:100E10000C94160F19A68091C1018FA3803529F477
:100E20009B8D91110C94180F7AC2AF8DA23009F0EE
:100E300076C2BFA1B11104C0EB8DE11170C22AC00E
:100E400020E030E0A9016091CC017091CD0180914A
:100E5000CE019091CF010E94CB36882309F4EAC7D6
:100E6000FFA1FC3809F445C240F4F230A9F0F33098
:100E7000B1F0F13009F053C20AC02FA12E3809F4A5
:100E800038C208F433C22F3809F430C248C23B8D4F
:100E9000311145C21F8E43C24BA144604BA38B8DC1
:100EA000882309F4DFCDBBADAB2FB0E0B8ABAFA763
:100EB000FDADEF2FF0E0FCABEBAB81E090E07C010F
:100EC0000BAC02C0EE0CFF1C0A94E2F70DAC02C0A2
:100ED000880F991F0A94E2F7E82AF92A2B8D822FAE
:100EE00090E08E219F21892B09F4A6C7FD01EE0F0A
:100EF000FF1FEE0FFF1FE054FE4FAA0FBB1FAA0FEC
:100F0000BB1FA856BE4F2D913D914D915C9166A59A
:100F100077A580A991A90E94D5352B013C01EBA9A9
:100F2000FCA9EE0FFF1FEE0FFF1FE054FE4FABA911
:100F3000BCA9AA0FBB1FAA0FBB1FA856BE4F2D915D
:100F40003D914D915C9166A577A580A991A90E94DC
:100F5000D5354B015C01610130E8C322DD2427FE59
:100F6000F5C0E89427F84CE050E06EEE71E088E9B7
:100F700091E00E94983A892B11F481E27DC780911B
:100F8000C3018130B1F423E333E34BEC51E46091CE
:100F9000E5017091E6018091E7019091E8010E94DE
:100FA0002D396093E5017093E6018093E7019093FA
:100FB000E8018091E5019091E601A091E701B091EF
:100FC000E8018FAB98AFA9AFBAAFA3019201C301FB
:100FD000B2010E942D3927966CAF7DAF8EAF9FAFC7
:100FE0002797A5019401C501B4010E942D392B96C4
:100FF0006CAF7DAF8EAF9FAF2B9720E030E040E825
:1010000050E46FA978AD89AD9AAD0E942D392FA912
:1010100038AD49AD5AAD0E942D3927962CAD3DAD66
:101020004EAD5FAD27970E94D5352B962CAD3DADCB
:101030004EAD5FAD2B970E94D5356B017C0120E052
:1010400030E0A9010E94CB3687FDF8C6C701B60182
:101050000E94CC396B017C012B962CAD3DAD4EAD81
:101060005FAD2B9727966CAD7DAD8EAD9FAD27976D
:101070000E94D6350E94CC399B01AC01C701B60154
:1010800090580E94D5366B017C019FA1933021F4CA
:10109000F7FAF094F7F8F09420E030E0A9016FA996
:1010A00078AD89AD9AAD0E94CB3687FF11C0F7FAB3
:1010B000F094F7F8F0948FA998ADA9ADBAADB058F7
:1010C0008093E5019093E601A093E701B093E801D6
:1010D0000FA518A9000F111F000F111F00531E4F5D
:1010E000A7019601C501B4010E942D399B01AC01F5
:1010F000C301B2010E94D53520E030E040E05FE35B
:101100000E942D39D8016D937D938D939C931397F5
:101110000BA91CA9000F111F000F111F00531E4F18
:10112000A7019601C301B2010E942D39A5019401C6
:101130000E94D63520E030E040E05FE30E942D3988
:10114000F8016083718382839383E9C0212F30E0AB
:1011500038AF2FABE222F322EF2809F471C631EF4A
:1011600023228091C301813009F47BC0EFA5F8A947
:10117000EE0FFF1FEE0FFF1FE053FE4FC080D18028
:10118000E280F380A7019601C301B2010E94D53528
:101190002B013C01EBA9FCA9EE0FFF1FEE0FFF1F77
:1011A000E053FE4F80819181A281B3818FA798ABDC
:1011B000A9ABBAAB9C01AD01C501B4010E94D53504
:1011C0004B015C01A3019201C301B2010E942D39C0
:1011D0002B013C01A5019401C501B4010E942D39E8
:1011E0009B01AC01C301B2010E94D6350E94CC39EB
:1011F0004B015C01A7019601C701B6010E942D3980
:101200006B017C012FA538A949A95AA9CA01B901C6
:101210000E942D399B01AC01C701B6010E94D63551
:101220000E94CC396B017C016093E5017093E6016B
:101230008093E7019093E8019B01AC01C501B401E3
:101240000E94D5354B015C01E894B7F82AE037EDF0
:1012500043EA5BE3C501B4010E94ED3818164CF176
:101260005EC000EC11E08FA998AD0C2C02C09595E2
:1012700087950A94E2F780FF12C023E333E34BEC37
:1012800051E4D80150966D917D918D919C91539729
:101290000E942D39F801608B718B828B938BFFEF4D
:1012A000CF1ADF0A0C5F1F4F23E0C216D104D9F614
:1012B0005DCF20E030E040E05FE3C501B4010E9473
:1012C000ED3818160CF459CE2FE632E143E85AE314
:1012D000C701B6010E942D399B01AC01C501B401C3
:1012E0000E94ED3818160CF448CE19C03BA13061AD
:1012F0003BA38FA18E58823018F44BA148604BA3BA
:101300008B8D882309F4AECB4CE050E06EEE71E09B
:1013100088E991E00E94983A892B09F42ECE2BA1FE
:1013200021709BA190FF03C0C1018E7D03C0C1014C
:101330008E7D9C7FAF8DA111937E892B09F082C594
:101340008E01035F1F4F89E0F80111928A95E9F73A
:10135000222309F44BC08BA59CA5867B892B09F021
:1013600073C58091C001853311F081116DC58091E5
:101370008B0190918C01A0918D01B0918E01898B90
:101380009A8BAB8BBC8B9091890180918801892BC2
:101390004091CC015091CD016091CE017091CF016F
:1013A0004D875E876F87788B84608D8B809170010D
:1013B00085FF06C08EEE91E00E94E42A811146C5A9
:1013C000B8018EEE91E00E94560F80911A018111B2
:1013D00041C50E94AB1C892B09F43CC580E2809377
:1013E0001A010E94BE1E0E94CD1734C58091700163
:1013F000F090890181FF26C08FA18150833018F0C1
:10140000FBA1F064FBA32B8D222339F03F8D3230FA
:1014100021F44BA140684BA315C080E1F81212C023
:101420008091800181509BA19074833030F4992386
:1014300049F09BA190629BA305C0911103C0ABA191
:10144000A062ABA38091DD019091DE01A091DF014C
:10145000B091E0018093940190939501A09396013F
:10146000B09397018091C20180938101882311F08C
:1014700088E08D8B8091CC019091CD01A091CE011F
:10148000B091CF0180938F0190939001A09391012F
:10149000B09392018D879E87AF87B88B8090E901CA
:1014A0009090EA01A090EB01B090EC01A5019401AD
:1014B00060918B0170918C0180918D0190918E01D2
:1014C0000E94CB36BBA1B074EB2E811103C0EBA1FF
:1014D000E5FF20C0FF2071F0FBA1F7FD0BC0EE205F
:1014E00021F040E050E0BA0102C0B501A4018F2D07
:1014F0000E940A348091E9019091EA01A091EB01E8
:10150000B091EC0180938B0190938C01A0938D019D
:10151000B0938E01E1100CC080918B0190918C01F1
:10152000A0918D01B0918E01898B9A8BAB8BBC8B76
:101530008091ED01809393018091CA01909189017E
:10154000981751F049895A896B897C890E940A341D
:101550008091CA01809389019D8980918901892B9D
:101560008D8BF090C901809188018F15A9F0809131
:101570001A01823029F00E94F9338F2D0E94253202
:101580008091C901811103C01092880105C090911A
:101590008801892B809388019D8980918801892BFE
:1015A0008D8B8091C001843099F4C090E101D0907E
:1015B000E201E090E301F090E40180911A018230B1
:1015C00039F00E94F93340E0C701B6010E9497311B
:1015D0008091C501809384018091C3018093820131
:1015E0002F8D233071F58091C60180938501811183
:1015F00008C01092F6011092F7011092F8011092B3
:10160000F901C090F601D090F701E090F801F09058
:10161000F901A70196016091BC017091BD01809113
:10162000BE019091BF010E94CB36882351F0C09239
:10163000BC01D092BD01E092BE01F092BF010E94B8
:101640005E2B8091C70190918601981769F0809375
:1016500086018CE0FE013196A4EAB1E001900D9282
:101660008A95E1F70E945E2B8091C40180938301EB
:101670008091C0018632F1F138F48C3109F18E315C
:10168000F9F08A3069F04FC08C35D1F1863609F413
:1016900041C0883209F047C068E971E087E02DC099
:1016A00060ED71E089A50E94161D8091860139A523
:1016B000381339C08CE0E0EDF1E0A4EAB1E025C0D8
:1016C0008D8981608D8B4F8D442329F0B8018EEE7A
:1016D00091E00E94560FB80180ED91E00E94560FF4
:1016E0008CE0E0EDF1E0A8E9B1E001900D928A957F
:1016F000E1F719C068E971E086E00E94161D13C089
:101700008CE0EEEEF1E0A0EBB1E001900D928A9555
:10171000E1F707C08CE0E0EBF1E0DF011D928A9574
:10172000E9F70E945E2B8091C10180938001803592
:1017300009F41CC3BF8DB23009F018C3813021F405
:10174000BE01635F7F4F06C0811109C08D89816032
:101750008D8BB8018EEE91E00E94560FFEC2825032
:10176000823008F093C28091E5019091E601A0914A
:10177000E701B091E8018F8F98A3A9A3BAA3ABADFD
:1017800094E0A99F70011124F701E856FE4FF8A7D5
:10179000EFA3970120533E4F3AA729A7D9014D90B7
:1017A0005D906D907C902081318142815381C30195
:1017B000B2010E94D6356BA77CA78DA79EA7EDAD81
:1017C000B4E0EB9F80011124980128563E4F3CAFB6
:1017D0002BAFC80180539E4F9EAF8DAFDC018D9023
:1017E0009D90AD90BC90F90120813181428153815F
:1017F000C501B4010E94D6356FA778AB89AB9AAB0F
:1018000077FA709477F87094D501C401B0588B8F33
:101810009C8FAD8FBE8FF701E251FE4F2BA53CA5EB
:101820004DA55EA560817181828193810E94D5352D
:101830006B017C01F801E251FE4F2FA538A949A99F
:101840005AA960817181828193810E94D5354B01B3
:101850005C01A7019601C301B2010E942D396BAB57
:101860007CAB8DAB9EABA50194016B8D7C8D8D8D7A
:101870009E8D0E942D399B01AC016BA97CA98DA97D
:101880009EA90E94D6356BAB7CAB8DAB9EABA50100
:101890009401C301B2010E942D394B015C01A701E3
:1018A00096016B8D7C8D8D8D9E8D0E942D399B01B7
:1018B000AC01C501B4010E94D5352BA93CA94DA9A5
:1018C0005EA90E9455366B017C019BA192FF13C05B
:1018D0002DEB37E346E055EBC701B6010E94ED382A
:1018E00087FD1DC02BED3FE049EC50E4C701B60178
:1018F0000E94D53512C02DEB37E346E055E3C70112
:10190000B6010E94CB36181654F02BED3FE049EC9F
:1019100050E4C701B6010E94D6356B017C0180906E
:10192000640190906501A0906601B09067012F8DD1
:1019300038A149A15AA1CA01B9010E94D635A50111
:1019400094010E94D535A50194010E942D390E9471
:10195000CC394B015C0120E030E040E05FE3C7019F
:10196000B6010E942D392F8D38A149A15AA10E949C
:101970002D399F77A50194010E94D5360E94BA3770
:101980000E944E377CAB6BABDB01AB2B09F4D8CE9E
:101990001D894B01A12CB12C13FF12C0C501B4014C
:1019A0000E947D379B01AC016D857E858F8598896E
:1019B0000E942D396D877E878F87988B177F1D8BAF
:1019C000C501B4010E947D374B015C019B01AC0154
:1019D000C701B6010E94D5366BA37CA38DA39EA33D
:1019E000EFADB4E0EB9FC00111248C0108561E4FEF
:1019F000FC01E251FE4FD8012D913D914D915C913A
:101A000060817181828193810E94D535A501940105
:101A10000E94D53627966CAF7DAF8EAF9FAF2797CC
:101A20002BA13CA14DA15EA1CA01B9010E942D3993
:101A30009B01AC0160E070E080E090E40E94D5354D
:101A40006B017C012BEA3AEA4AE25EE36BA17CA1DE
:101A50008DA19EA10E942D394B015C0120E030E058
:101A600040E850E4C701B6010E94D6359B01AC01A5
:101A7000C501B4010E942D396FAB78AF89AF9AAF21
:101A800020E030E040E05FE3C701B6010E942D395D
:101A900023966CAF7DAF8EAF9FAF23971F8E22240E
:101AA0002394312CEBA9FCA9E215F30509F448CEE7
:101AB000BF8DBC3008F044C02B8D3C8D4D8D5E8DAC
:101AC00023966CAD7DAD8EAD9FAD23970E942D39D1
:101AD0006B017C01A30192016FA978AD89AD9AAD2C
:101AE0000E942D39A70196010E94D6357B016C0119
:101AF000A301920123966CAD7DAD8EAD9FAD239772
:101B00000E942D394B015C012B8D3C8D4D8D5E8DDE
:101B10006FA978AD89AD9AAD0E942D399B01AC01BA
:101B2000C501B4010E94D5352B013C01EF8DEF5F5B
:101B3000EF8F470156018B8E9C8EAD8EBE8E65C099
:101B4000B10180E090E00E947D372BA13CA14DA126
:101B50005EA10E942D396B017C010E94D0366B8FF3
:101B60007C8F8D8F9E8FC701B6010E94BE394B01BD
:101B70005C01A9A5BAA5CD90DD90ED90FC90F7FA97
:101B8000F094F7F8F094ADADBEAD8D919D910D90B0
:101B9000BC91A02D8F8F98A3A9A3BAA3A7019601EA
:101BA0006B8D7C8D8D8D9E8D0E942D392B013C017E
:101BB0002F8D38A149A15AA1C501B4010E942D3928
:101BC0009B01AC01C301B2010E94D6352B013C013F
:101BD000A7019601C501B4010E942D396B017C015A
:101BE0002F8D38A149A15AA16B8D7C8D8D8D9E8D35
:101BF0000E942D399B01AC01C701B6010E94D53569
:101C00006B8F7C8F8D8F9E8F1F8EA30192016BA592
:101C10007CA58DA59EA50E94D635EFA1F8A5608371
:101C20007183828393832B8D3C8D4D8D5E8D6FA54B
:101C300078A989A99AA90E94D635ABADBCAD6D93A0
:101C40007D938D939C93139727962CAD3DAD4EAD10
:101C50005FAD2797F80160817181828193810E9435
:101C6000D635D8016D937D938D939C931397BE01C8
:101C7000635F7F4F88E991E00E94560F80911B01BE
:101C800081116BC0BFEF2B1A3B0A0CCF8D8984608A
:101C90008D8B80911A01823009F45FC00E94F93364
:101CA00080911B01811162C0FBA1F071FF2E109287
:101CB0001F012BA123FB882780F90E94AA2B86B144
:101CC000807290910001891749F084E00E94CB2A2C
:101CD0000E94ED3280E00E94AA2B48C0B8018EEE2F
:101CE00091E00E94560F81E08093190182E00E94EA
:101CF000DB2A0E94ED3280911B01811137C0809157
:101D00001A018111F6CF80911901813081F4FF20F1
:101D100051F08CE0E1E0F1E0ADE0B1E001900D9236
:101D20008A95E1F707C085E00E94CB2A03C081E0D5
:101D300080931F011092190180E00E94AA2B0E943B
:101D4000ED320E94572A0E94BB1C0E94C6310E949D
:101D5000562E80911F0181118CC08CE0EEEEF1E0D7
:101D6000A8E9B1E001900D928A95E1F78091C80150
:101D700080938701882309F47FC00E94F933809102
:101D8000870190911A01833041F49230D1F188E0BB
:101D90000E94DB2A0E94ED3234C081E080938001F2
:101DA0001092840110928301109281011092860199
:101DB000109289011092880184E68093210180931A
:101DC000220180932301923091F064EA71E080E077
:101DD0000E949D1E8823E1F10E945E2B40E050E0AE
:101DE000BA0180E00E94C13280E00E94253281EF7A
:101DF00091E00E94B62C88E891E00E94B62C0E94E7
:101E0000512E109287012FC081E036C082E034C08D
:101E100088E132C086E230C089E12EC084E02CC067
:101E20008BE12AC085E228C084E126C08EE124C06F
:101E30008FE122C086E120C080E21EC082E21CC089
:101E400083E21AC084E218C080E116C08FE014C09B
:101E500087E012C08CE0EEEEF1E0A8E9B1E001907D
:101E60000D928A95E1F780E007C01A8E1BA20C94B0
:101E7000DF010E945B347ACFC65BDF4F0FB6F89468
:101E8000DEBF0FBECDBFDF91CF911F910F91FF90AD
:101E9000EF90DF90CF90BF90AF909F908F907F900A
:101EA0006F905F904F903F902F900895FF920F9307
:101EB0001F93CF93DF938C01EB018091700185FF1D
:101EC00026C0F0901A0180E2F81629F1C8010E949C
:101ED000E42A8823E1F081E080931D0188E0F81670
:101EE00041F00E94613482E00E94CB2A0E94ED32D0
:101EF0000EC088E00E94DB2A0E94ED3280911B0117
:101F0000811105C080911A018111F6CFEACF80912D
:101F10001A01823041F10E94ED3280911B01811142
:101F200022C09091DA028091D902981303C00E94D6
:101F3000D731F1CFBE01C8010E949727811113C08C
:101F40008091700181FF0FC0888584FF0CC04C8197
:101F50005D816E817F8180E1DF91CF911F910F9133
:101F6000FF900C940A34DF91CF911F910F91FF9055
:101F70000895CF93DF93CDB7DEB761970FB6F8948E
:101F8000DEBF0FBECDBF8091C00082608093C000D5
:101F90001092C50080E18093C4008091C1008869DF
:101FA0008093C10080E090E00E94511E8A3009F0C9
:101FB0003CC545E550E061E070E08BE291E00E94B5
:101FC000591E892B09F431C58AB18C618AB9209ACE
:101FD0008AB1806E8AB9809181008F7E8093810062
:101FE00080918100886080938100809180008C7F47
:101FF00080938000809180008F708093800080911A
:102000006E00887F80936E0014BC15BC80916E00BA
:10201000816080936E0087B1887F87B988B18760BF
:1020200088B980916C00876080936C008091680013
:102030008260809368008CE0E1E0F1E0DF011D92B6
:102040008A95E9F7789410921A018091700184FFC3
:1020500003C081E080931A01AAE12A2EA1E03A2E62
:102060009924939480911A0191E1F10111929A952A
:10207000E9F780931A0184E680932101809322017D
:10208000809323018CE0ADE0B1E01D928A95E9F7E1
:102090001092190110921D0610921E0610921F0632
:1020A000109220068091FA018093FB0180E4E0E821
:1020B000F1E011928A95E9F764EA71E080E00E940C
:1020C0009D1E811103C087E00E94C92C0E94283404
:1020D0003B9A43980E94C3303D98459A80E00E9405
:1020E000AA2B0E94BB1C0E94572A0E94C6310E9444
:1020F0005B3487EF91E00E94B62C8091700183FFE2
:1021000010C00E94AF2E882361F090921A0181EFD7
:1021100091E00E94B62C80E991E00E94B62C0E94CA
:10212000512E80911A01817899F081EF91E00E94FF
:10213000B62C8BEC91E00E94B62C0E94512E90920E
:102140001A0110E000E0E2E0EE2EF4E08F2E29C04C
:1021500010921A010E94DD2CF4CFE92FF0E0EF5D20
:10216000F94F80819F5F913809F490E09093FB01D3
:102170008F3FE9F08A3021F50E94ED3280911B01FA
:10218000811170CFE12FF0E0EF5EF84F1082F02F59
:10219000F170FF2E00FF18C08BE00E94C92C10E0E8
:1021A00000E09091FB018091FA019813D6CF0E9434
:1021B000D7310E94ED3280911B01882391F352CFD9
:1021C0008D3009F00CC4D8CF80911107882309F411
:1021D00003C4843209F0F8C3998A809112078334CA
:1021E00009F134F4882361F0843209F006C11AC081
:1021F0008A3459F08835B1F0873409F0FEC012C036
:102200008FE592E00E94B62CDDC380911A018F7D8C
:1022100009F0C8C3809113078D3309F0CBC30E9426
:10222000A501C3C3909113079111C4C3833409F46A
:10223000B2C01CF4843239F0C5C3873469F08835E4
:1022400009F4C9C0BFC380911A018871F82E09F042
:10225000A9C30E943F2DB6C389E592E00E94B62C27
:10226000809180018C3838F085E592E00E94B62C90
:10227000809180018A580E94902C86E492E00E940E
:10228000B62C809186018A5C0E94902C86E492E0B4
:102290000E94B62C809184018F5E0E94902C86E46F
:1022A00092E00E94B62C8091820125E1281B822FAA
:1022B0000E94902C86E492E00E94B62C80918301CB
:1022C000865A0E94902C86E492E00E94B62C80915F
:1022D00081019EE5981B892F0E94902C8091870197
:1022E000882399F089E492E00E94B62C80918701BE
:1022F000833029F08E3139F0823039F404C080E324
:102300000E94093202C00E94902C89E492E00E944F
:10231000B62C80918901803131F0803231F0811109
:1023200007C085E303C083E301C084E30E94093250
:1023300089E492E00E94B62C80918801882311F0F4
:1023400088E301C089E30E94093282E592E00E949D
:10235000B62C809193010E94902C8FE492E00E9411
:10236000B62C60918F0170919001809191019091B4
:1023700092010E94592C8CE492E00E94B62C60914C
:102380008B0170918C0180918D0190918E0140E0C4
:102390000E94BC2B0EC080911A01823069F40E9409
:1023A000613481EF91E00E94B62C88EA91E00E94AE
:1023B000B62C0E94512E06C38111F4C2E0921A017C
:1023C00081EF91E00E94B62C81EB91E00E94B62C47
:1023D0000E94512E3BC080911A01813009F0F2C257
:1023E00081EF91E00E94B62C89EB91E00E94B62C1F
:1023F0000E94512E10921A01E5C290911A0192305A
:1024000008F0D0C2893409F49DC034F4833271F0ED
:10241000883409F45AC045C1823509F4ECC08335CB
:1024200009F47EC08E3409F03CC115C180911307B8
:102430008111C0C210E0BE016F5F7F4F812F0E94EB
:102440009D1E811105C087E00E94C92CF12CBAC2E3
:1024500083E492E00E94B62C163029F0173041F444
:102460008DE392E002C080E492E00E94B62C04C0AA
:1024700086E3810F0E94902C8AE30E940932CE01EC
:1024800001960E94772C0E94512E1F5F183099F6FA
:1024900087E392E00E94B62C80EB91E00E94772CBB
:1024A0000E94512E81E392E00E94B62C6091BC0103
:1024B0007091BD018091BE019091BF010E94682C76
:1024C0000E94512E0E94562E7DC28091700184FF81
:1024D00066C280921A0180911307882381F090913F
:1024E0001407911167C2893539F08A3539F088357A
:1024F00009F060C281E003C082E001C084E00E9474
:10250000073580911B0181115DC210921A010E9452
:102510004F1580911307811155C20E94DD2C96CF73
:10252000809113078C3409F045C2809114078035DF
:1025300009F040C28091150781113CC280E80E94D9
:10254000DB2A40C2E98A80911307811136C040E539
:1025500050E06EEA73E081E197E00E94591E892BFA
:1025600051F41092110740E550E061E177E08EEA06
:1025700093E00E94CC1C8DE192E00E94B62C0E9458
:102580008A2A0E94512E87E192E00E94B62C81E5B2
:102590000E94093286E50E94093288E40E940932CD
:1025A0008CE20E9409328FE00E94902C8CE20E9403
:1025B000093280E80E94902CFCCEA3E0A98B8D33D9
:1025C00009F0F8C183E0282F30E0F901EF5EF84F01
:1025D0009081D901A25FB84F9C938F5F9081911138
:1025E000F2CF898B40E550E061E177E08EEA93E03D
:1025F0000E94CC1CE7C180911307833509F0DAC132
:1026000080911407843509F0D5C1809115078D3369
:1026100009F0D0C1809117078111CCC180911607B4
:10262000843239F08A3239F0833209F0C3C182E052
:1026300003C081E001C08FEF0E942A1D81EF91E06D
:102640000E94B62C85E791E00E94B62C0E94512E84
:102650000E946134B7C1E98A8091130781111DC0BE
:1026600010E0812F0E94972A811104C087E00E9408
:10267000C92C0EC084E192E00E94B62C812F0E94EA
:10268000902C8DE30E9409320E948A2A0E94C52C58
:102690001F5F123009F496C1E4CF911183C111E09C
:1026A00001C010E0BE01635F7F4FCE0141960E94E2
:1026B0002135811103C072E0F72E84C1E98981E0E0
:1026C0008E0F898BF0E0EF5EF84F90819D3309F01B
:1026D00071C1112371F1482F50E0282F30E0F9012A
:1026E000EF5EF84F9081241B350BD901AF5EB84FD8
:1026F0009C938F5F90819111F0CF898B0E94A501EF
:10270000811153C16D857E858F8598890E94103A0D
:102710000E944E37162F0E94F933B1E51B9FC0016E
:10272000112440E550E061E177E09D5F0E94CC1C00
:102730008DCEBE016F5F7F4FCE0141960E94213545
:10274000882309F4B8CFE989F0E0EF5EF84F808183
:10275000811130C1AD84BE84CF84D88820E030E0C0
:102760004FE753E4C601B5010E94ED3818160CF48A
:1027700021C149805A806B807C80C601B5010E94CE
:102780004E37062F20E030E0A901C301B2010E94BC
:10279000CB3687FD0CC1043608F440C0045680E0F7
:1027A000033098F510E0000F111F000F111F823049
:1027B00079F0F801833011F1813019F0E55DFE4FB9
:1027C00002C0E95CFE4F4082518262827382E4C0A3
:1027D0000D5B1E4F20E030E040E752E4C301B20140
:1027E0000E942D3920E030E040E752E40E942D396C
:1027F000F8016083718382839383CEC0E15BFE4FD7
:1028000077FA709477F87094DECF8F5F0A3008F40F
:10281000D1C0843009F4CEC00A50C2CFC301B20186
:102820000E94103A0E944E3710E00132110508F064
:10283000C1C0F801E75BFF4F0C94783A633008F4AD
:10284000BCC060935B01A8C060935E01A5C06093AB
:102850005C0102C060935D010E941E159DC08091C5
:102860007001662311F0846095C08B7F93C08091C6
:102870007001662311F080648DC08F7B8BC08091C6
:102880007001662311F0806801C08F77809370011A
:1028900080E00E94AA2B80C060935F017DC04092BF
:1028A000600150926101609262017092630174C094
:1028B00040926401509265016092660170926701D6
:1028C0006BC080917001662311F0816001C08E7F22
:1028D000809370010E945E2B5FC08091700166231F
:1028E00021F084FF6DC0806255C08F7D53C0809100
:1028F0007001662311F0886001C0877F80937001AA
:102900000E94C33049C080917001662311F080613C
:1029100041C08F7C3FC0609371013EC04092720104
:1029200050927301609274017092750135C04092AB
:1029300076015092770160927801709279012CC0F3
:1029400070E070937B0160937A0126C040927C0115
:1029500050927D0160927E0170927F011DC0409275
:1029600068015092690160926A0170926B0108C01F
:1029700040926C0150926D0160926E0170926F01F5
:102980000E94283409C080917001662311F0826092
:1029900001C08D7F809370010E94091D13C055E016
:1029A000F52E10C048E0F42E0DC0F82E0BC034E018
:1029B000F32E08C023E0F22E05C096E0F92E02C0E7
:1029C0008AE0F82E8F2D08C080911A01817211F0D3
:1029D00089E0E3CB0E94A5010E94D52CE0CB002327
:1029E00029F0893209F0DDCB0D7FDBCB813208F491
:1029F000D8CB8F3209F4D5CB883289F08B3389F06C
:102A00001F3488F4212F30E01F5F9FE9980FF901F0
:102A1000EF5EF84F9A3108F480528083C2CB02E017
:102A2000C0CB04E0BECB01E0BCCB87E00E94C92C48
:102A30008FEF0E942A1D0E943F2DC6CA80915C0123
:102A4000682F20915D01422F982F917080FD94E0B6
:102A5000822F817020FD80E261FD986041FD8064DD
:102A600062FD906142FD80689093FC018093FD01BE
:102A700008951F920F920FB60F9211248F939F9378
:102A80008BB19091FC019C71837E892B8BB915BC15
:102A90009F918F910F900FBE0F901F90189580916E
:102AA0006F008D7F80936F0080918100887F8160AF
:102AB000809381001092FE0180915E0190911A0135
:102AC0008F3F39F420911E06211103C0903881F404
:102AD00002C0943069F090E0009741F0EFE9FFE028
:102AE0003197F1F700C000000197F6CF81E001C0F7
:102AF00080E09091700192FF02C091E089278823C5
:102B000011F0289A0895289808951F920F920FB6F1
:102B10000F9211242F933F934F935F936F937F9363
:102B20008F939F93AF93BF93EF93FF938091FE0199
:102B3000811122C28BB190910E02907E8F71892BF0
:102B40008BB98BB1837E90910D02892B8BB98091CB
:102B50000C0286BD82E085BD81E08093FE01789401
:102B60008091200290912102892B09F0BFC08091B1
:102B7000220290914D02981709F4A4C0E09122021C
:102B80002E2F30E087E0E89FF0011124ED5DFD4F2E
:102B9000F0932102E0932002828193819093890037
:102BA000809388008081918190931C0280931B0206
:102BB000E48180911D028E1761F1E0931D0282E194
:102BC000E89FF0011124E25BFD4FF0931F02E093B8
:102BD0001E0284859585A685B785B695A795979598
:102BE00087958093070290930802A0930902B093FF
:102BF0000A028093030290930402A0930502B0930B
:102C000006028093FF0190930002A0930102B0930B
:102C10000202A0911E02B0911F0250969C91509703
:102C20008091FD01892780930E0287E0829FF00149
:102C3000839FF00D1124ED5DFD4F25814D915D9138
:102C40006D917C911397022E04C0769567955795E8
:102C500047950A94D2F740930F0250931002609365
:102C600011027093120214964D915D916D917C91B9
:102C70001797022E04C076956795579547950A9445
:102C8000D2F740931302509314026093150270938D
:102C9000160218968D919D910D90BC91A02D04C0A7
:102CA000B695A795979587952A95D2F780931702A1
:102CB00090931802A0931902B0931A0286810E9481
:102CC000B33214C00E944F15E0911E02F0911F0212
:102CD0008189882339F01092B3008091B0008F77FA
:102CE0008093B00084E00E94DB2A46C180911901E4
:102CF0008130B1F486B1807290910001891781F022
:102D0000109219018CE0E1E0F1E0ADE0B1E001905A
:102D10000D928A95E1F780911D06806480931D06CF
:102D200010920D024091FF0150910002609101024A
:102D30007091020280910F0290911002A0911102F5
:102D4000B0911202840F951FA61FB71F8093FF0139
:102D500090930002A0930102B0930202E0911E0240
:102D6000F0911F0244855585668577854817590778
:102D70006A077B0768F524E020930D02448555859A
:102D800066857785841B950BA60BB70B8093FF0197
:102D900090930002A0930102B093020220898091D7
:102DA000010190910201A0910301B091040125FF5E
:102DB00004C00197A109B10903C00196A11DB11D6D
:102DC0008093010190930201A0930301B093040149
:102DD0004091030250910402609105027091060235
:102DE0008091130290911402A0911502B0911602E5
:102DF000840F951FA61FB71F8093030290930402B0
:102E0000A0930502B09306024485558566857785B3
:102E1000481759076A077B0778F520910D0228604B
:102E200020930D024485558566857785841B950B17
:102E3000A60BB70B8093030290930402A0930502A4
:102E4000B093060220898091050190910601A0911E
:102E50000701B091080126FF04C00197A109B1093B
:102E600003C00196A11DB11D809305019093060139
:102E7000A0930701B0930801409107025091080206
:102E80006091090270910A028091170290911802D4
:102E9000A0911902B0911A02840F951FA61FB71FA7
:102EA0008093070290930802A0930902B0930A024C
:102EB0004485558566857785481759076A077B07D6
:102EC00078F520910D02206120930D0244855585EF
:102ED00066857785841B950BA60BB70B809307023D
:102EE00090930802A0930902B0930A02208980916E
:102EF000090190910A01A0910B01B0910C0127FFEB
:102F000004C00197A109B10903C00196A11DB11D1B
:102F10008093090190930A01A0930B01B0930C01D7
:102F200080911A01843039F490910D028091200132
:102F3000892380930D0280911B0290911C020197BE
:102F400090931C0280931B02892B69F4109221023A
:102F500010922002809122028F5F8093220286309D
:102F600011F41092220290910D028091FC018927A8
:102F700080930D021092FE01FF91EF91BF91AF91EE
:102F80009F918F917F916F915F914F913F912F9181
:102F90000F900FBE0F901F9018958091700182FFC7
:102FA00002C0289A01C028988091FC0180930D02EC
:102FB00080915B01880F8450819580930C028091F1
:102FC0006F00826080936F0008953F924F925F92EE
:102FD0006F927F928F929F92AF92BF92CF92DF9229
:102FE000EF92FF920F931F93CF93DF93CDB7DEB78E
:102FF000A4970FB6F894DEBF0FBECDBF10911E068A
:10300000112391F181E080931A0189EA92E00E94F4
:10301000B62C812F0E94902C0E94C52C85EF91E048
:10302000019739F0EFE9FFE03197F1F700C00000B8
:10303000F7CF1150123030F08FB7F89410921E066F
:103040008FBF12C081EF91E00E94B62C8FED91E00E
:103050000E94B62C0E94512E80E10E94D12A8091BC
:103060001D0684FFFCCFE8CF10911D06112309F443
:10307000BBC214FF04C081E080931B01BFC310FFDB
:10308000BFC18CE0E1E0F1E0DE01599601900D92C4
:103090008A95E1F7BE01675E7F4FCE010D960E94D3
:1030A000222B8CE30E94093280911A018830E1F0D2
:1030B00058F4813099F1A8F0823099F1843009F008
:1030C00043C084EF92E03EC0803229F118F4803191
:1030D00071F03AC0803441F18038B1F58CED92E066
:1030E00031C087E093E02EC083E093E02BC0809155
:1030F0001C0187FD10C08DEF92E00E94B62C8091DC
:103100001C0180FF06C080E31AC082FF17C085FF44
:10311000FACF81E314C089EF92E014C08EEE92E002
:1031200011C088EE92E00EC082EE92E00E94B62CB2
:1031300080911C0183FFE9CF83E301C082E30E94F9
:10314000093202C00E94B62C80915F01F82FF17005
:10315000BF2E80FF07C080912601882319F085EDDE
:1031600092E053C04090BC015090BD016090BE0100
:103170007090BF0144EA842E41E0942E9E012F5F9F
:103180003F4F7901CE010D966C0100E0F401619191
:103190007191819191914F012085318542855385AF
:1031A0000E94D635F7016083718382839383023056
:1031B00061F4A30192010E94D635F7016083718307
:1031C00082839383BB2019F0CACFB11011C0F701DD
:1031D0002081318142815381F60160817181828138
:1031E00093810E94D535F601608371838283938336
:1031F0000F5FF4E0EF0EF11C24E0C20ED11C03308F
:1032000029F6B110ACCF8EEC92E00E94B62CCE0124
:103210000D960E94772C80915F0181FF1FC089EC81
:1032200092E00E94B62C9091FB058091DA029817EB
:1032300010F0815F01C08150891B0E94902C8CE2AC
:103240000E9409328091FB019091FA01981710F0C9
:10325000805801C08150891B0E94902C84EC92E020
:103260000E94B62C80911A018C7749F06091BF02C0
:103270007091C0028091C1029091C20203C060E0CF
:1032800070E0CB010E94592C8CE20E9409326091BF
:103290002701709128018091290190912A0140E035
:1032A0000E94BC2B0E94AF2EF82E0E94632B082F89
:1032B00086B1982F907280910001E92EE8268F2D1B
:1032C000802B8E2959F18FEB92E00E94B62CEE20D4
:1032D00019F080E50E940932FF2079F0F0FE03C06A
:1032E00088E50E940932F1FE03C089E50E94093297
:1032F000F2FE03C08AE50E940932002379F000FF44
:1033000003C082E50E94093201FF03C088E40E94E5
:10331000093202FF03C083E50E9409328091260131
:10332000882321F081508093260118C080911A01D2
:103330008C7711F08DE101C089E0809326018091A6
:103340002501811103C081E08093250189EB92E082
:103350000E94B62CCE0101960E94772C0091250187
:10336000002321F001500093250142C080911A01F1
:103370008C7711F083E101C089E08093250184EB13
:1033800092E00E94B62C809121010E94902C8CE248
:103390000E940932809122010E94902C8CE20E94AE
:1033A0000932809123010E94902C8091B00087FF08
:1033B00005C02D9B02C002E001C001E0439B03C099
:1033C000FF24F39403C0002399F0F12C80EB92E0EA
:1033D0000E94B62C002339F0013011F483E501C0BE
:1033E00083E40E940932FF2019F086E40E9409322A
:1033F0008EE30E9409320E94C52C81E00E94D12AEE
:10340000812F887E09F467C080911A01982F9370EC
:1034100009F050C08872A1F080911C01807C81F479
:103420000E942B2682E080931E0180911A01803237
:1034300039F417FDE1C180911C01806880931C0163
:1034400080911A01811103C091E090931C0116FF35
:1034500007C085FD05C090911C01906490931C01EC
:1034600013FF05C0807E19F480E180931A0115FFD7
:1034700021C081EF91E00E94B62C8DE991E00E947D
:10348000B62C0E94512E80911C0187FD0EC0909198
:103490001A01903439F483FFABC1837E826080933C
:1034A0001C01A6C1903809F0A3C180911C01806263
:1034B00080931C0117FF0CC080911A01813029F400
:1034C00080911C01856080931C0180E880931A0123
:1034D00088EE0E94D12A11FF44C0812F8876F1F531
:1034E00080911A01803471F480911C0185FD0AC01D
:1034F00084FF03C010921A0105C082FF03C08860D8
:1035000080931C0180911A01882381F084FF26C0DA
:1035100090911C0190FF22C0803141F480912401E0
:10352000882321F088608093240118C010921E0126
:103530000E94AB1C892B71F080911C0186FD0AC092
:1035400010921C0188E080931A010E94BE1E0E9406
:10355000CD1704C010921C0110921A0182E00E9443
:10356000D12A12FF41C080911A01807D90911C01E7
:103570008823D9F080911D01811117C097FD15C0D6
:103580000E942B268091DA028093D8020E944F2657
:1035900080911E0181FF05C090911C019160909364
:1035A0001C01897F80931E011CC097FF0AC01092E6
:1035B0001E010E94BB1C0E94572A0E945B340E947D
:1035C000C63180911C0185FF08C08F778160809390
:1035D0001C0180E480931A0104C010921C01109217
:1035E0001A0184E00E94D12A90911F06992309F4C0
:1035F000ABC08FB7F89410921F068FBF4091210186
:1036000090FD02C0842F01C084E691FD865F92FD8B
:103610008A5093FD8F5F94FD8150893C08F088ECBF
:103620008A3008F48AE03091220195FD02C0232FF0
:1036300001C024E696FD22E397FD29E1481303C06B
:10364000231709F481C08093210120932201109255
:1036500025011091DA023090FB0589E9D82E96E712
:10366000E92E26E9F22E0EE732E3432E131509F474
:1036700057C0812E912C489CC001499C900D11246B
:10368000FC01E552FD4F5F01CF010E94381C562E10
:10369000672E782EC92E2D2D3E2D4F2D502F0E9496
:1036A000ED3818164CF42D2D3E2D4F2D502F6D2D2D
:1036B0007E2D8F2D902F08C0252D362D472D5C2D6A
:1036C000652D762D872D9C2D0E942D39F501668B59
:1036D000778B808F918F489CC001499C900D11245D
:1036E0009C0125523D4F7901F90182A093A0A4A02D
:1036F000B5A0A501940166897789808D918D0E947E
:10370000ED3818162CF4F701868A978AA08EB18EB0
:103710001F5F103109F410E0D52C73010C2DA6CFDA
:103720008D2D9E2DAF2DB02F8093190690931A06E4
:10373000A0931B06B0931C060E942B268091DA02F0
:103740008093D8020E944F2690912006992309F475
:1037500048C08FB7F894109220068FBF20912301A4
:1037600090FD02C0822F01C084E691FD865F92FD2C
:103770008A5093FD8F5F94FD8150893C08F088EC5E
:103780008A3008F48AE0281749F020911E01286049
:1037900020931E01809323011092250180911A012C
:1037A00095FF0DC0803159F420912401211102C0F0
:1037B00022E003C020FF03C0246020932401907CFA
:1037C00081F0882311F0887161F01091880116FF53
:1037D00002C01F7B01C01064812F0E94253210930C
:1037E000880180911A018C7F49F00E94BE1E06C09C
:1037F00080E480931A0159CE80E229CEA4960FB6B8
:10380000F894DEBF0FBECDBFDF91CF911F910F9116
:10381000FF90EF90DF90CF90BF90AF909F908F90F0
:103820007F906F905F904F903F900895F894F99932
:10383000FECF92BD81BD81E08FBB80B58627482F2A
:10384000082E000C550B262F30E024233523232B84
:1038500039F06F3F19F060BD84E006C084E104C018
:10386000882321F060BD84E28FBBF99A7894089593
:10387000BF92CF92DF92EF92FF920F931F93CF935D
:10388000DF937C01FC0102A513A5D4A5C5A5818900
:1038900080FF18C06091220170E080E090E00E94FB
:1038A0007F372AE037ED43E25CE30E942D399B012C
:1038B000AC01B8018D2F9C2F0E942D398B01D82F80
:1038C000C92F2DC082FD17C06091210170E080E0FA
:1038D00090E00E947F372AE037ED43E25CE30E94EC
:1038E0002D399B01AC01B8018D2F9C2F0E942D39E1
:1038F0008B01D82FC92FF701B6A0C7A0D0A4F1A47F
:103900002B2D3C2D4D2D5F2DB8018D2F9C2F0E940E
:10391000ED38181624F40B2D1C2DDD2DCF2D20E0B5
:1039200030E040E85FE3B8018D2F9C2F0E94ED3816
:10393000181624F000E010E0D0E8CFE3B8018D2F96
:103940009C2FDF91CF911F910F91FF90EF90DF900F
:10395000CF90BF9008958091DA029091FB0598175F
:1039600039F022E3829FC001112485529D4F0895B2
:1039700080E090E008958CE1E1E0F6E0DF011D9247
:103980008A95E9F71092DA021092FB0581E08093A4
:10399000D9021092D80208959F92AF92BF92CF920F
:1039A000DF92EF92FF920F931F93CF93DF935C010F
:1039B0008A017B01E40EF51EEB01912C6C01C61A05
:1039C000D70ACE018C0D9D1DCE15DF0589F0911013
:1039D00008C0292D990C330B232F221F2227221FC9
:1039E00001C021E06991922E960E0E94161CE9CF2B
:1039F000692DC501800F911FDF91CF911F910F910C
:103A0000FF90EF90DF90CF90BF90AF909F900C947D
:103A1000161C6AE080E090E00E94161C45E550E02C
:103A20006BE271E081E090E00C94CC1C0F931F934B
:103A3000CF93C82F8B010E94F9332DE0C29FC001A4
:103A400011244CE050E0B8019E5FCF911F910F917F
:103A50000C94CC1CEF92FF920F931F93CF93DF93A4
:103A6000CDB7DEB72C970FB6F894DEBF0FBECDBF33
:103A7000182F80FFD5C08AE080935B0189E1809395
:103A80005E0110925C0110925D0181E080935F0104
:103A90008AE097EDA3E2BCE380936001909361011B
:103AA000A0936201B09363018FE692E1A3E0BBE3D0
:103AB0008093640190936501A0936601B0936701C0
:103AC00080E090E0AAE7B4E48093680190936901F4
:103AD000A0936A01B0936B0110926C0110926D017A
:103AE00010926E0110926F011092710180E090E0CF
:103AF000A8ECB1E48093720190937301A0937401D8
:103B0000B093750180E090E0AAEFB3E48093760172
:103B100090937701A0937801B09379012AEF30E078
:103B200030937B0120937A0140E050E060E87FE32E
:103B300040937C0150937D0160937E0170937F01DF
:103B40001092700140E050E06AE773E440932B016B
:103B500050932C0160932D0170932E0140932F01FF
:103B600050933001609331017093320140933301DF
:103B7000509334016093350170933601809337017F
:103B800090933801A0933901B0933A0180933B019F
:103B900090933C01A0933D01B0933E0180933F017F
:103BA00090934001A0934101B093420180E090EADC
:103BB000ACE0B7E48093430190934401A0934501A6
:103BC000B09346018093470190934801A093490127
:103BD000B0934A0180934B0190934C01A0934D0107
:103BE000B0934E0180E090E0A8E4B3EC80934F01E5
:103BF00090935001A0935101B093520180935301CF
:103C000090935401A0935501B093560180935701AE
:103C100090935801A0935901B0935A010E94091D35
:103C200011FF10C0CE0101967C018CE0F7011192CA
:103C30008A95E9F700E0B701802F0E94161D0F5FFB
:103C40000830C9F712FF14C060E080E093E00E94E2
:103C5000161C60E081E093E00E94161C60E081E5A4
:103C600093E00E94161C60E082E593E00E94161C1F
:103C700013FF0AC060E08EEA93E00E94161C60E029
:103C80008FEA93E00E94161C2C960FB6F894DEBFC4
:103C90000FBECDBFDF91CF911F910F91FF90EF909D
:103CA0000895F999FECF92BD81BD81E08FBB80B5AB
:103CB00008959F92AF92BF92CF92DF92EF92FF92C0
:103CC0000F931F93CF93DF935B018A017C01E40E76
:103CD000F51EEC01912C6B01C81AD90AC6018C0F94
:103CE0009D1FCE15DF0589F00E94511E911008C05E
:103CF000292D990C330B232F221F2227221F01C0AD
:103D000021E0982E920E8993E9CFC501800F911F73
:103D10000E94511E21E030E0981611F020E030E0C2
:103D2000C901DF91CF911F910F91FF90EF90DF902C
:103D3000CF90BF90AF909F9008951F93CF93DF9344
:103D4000182FEB018DE0189FB00111247E5F4CE02D
:103D500050E0CE010E94591E892B59F48CE0FE01DF
:103D600011928A95E9F7BE01812F0E94161D80E00D
:103D700001C081E0DF91CF911F9108952F923F9272
:103D80004F925F926F927F928F929F92AF92BF926B
:103D9000CF92DF92EF92FF920F931F93CF93DF9317
:103DA000CDB7DEB7EF970FB6F894DEBF0FBECDBF2D
:103DB00080911E0180FD36C7909122028091FC0502
:103DC000981709F42FC78091FF0590910006892B61
:103DD00009F015C310911E0112FF09C08091FB0567
:103DE00022E3289FC001112485529D4F02C00E94EA
:103DF000AB1C909300068093FF052090FF05309048
:103E000000062114310409F40DC70091A902802F86
:103E1000817000FF03C01092A902EAC09091A8022D
:103E20009F5F953009F0892F8093A802E82EF12C2E
:103E300032E13E9DF0013F9DF00D1124E25BFD4F0C
:103E4000F093FE05E093FD05D10150969C915097AB
:103E5000908BE2E18E9FC001112420E030E04D9173
:103E60005D916D917D91F901E80FF91FE25BFD4FC6
:103E7000689412F8440F551F661F771F1694D1F7E8
:103E800040835183628373832C5F3F4F2C30310515
:103E900031F722E12E9DF0012F9DF00D11249F019D
:103EA000225B3D4FF10184859585A685B78543E06A
:103EB000880F991FAA1FBB1F4A95D1F7F901848764
:103EC0009587A687B787D1011C966D917D918D91BD
:103ED0009C911F970E947D376093AE027093AF0252
:103EE0008093B0029093B102F101268D378D40A1ED
:103EF00051A10E94D5369B01AC016093B202709330
:103F0000B3028093B4029093B50260E070E080EA5F
:103F10009FE30E94D5366093B6027093B7028093F8
:103F2000B8029093B9021092AA021092AB021092BA
:103F3000AC021092AD0211FD02C003FF1FC06091E0
:103F4000C7027091C8028091C9029091CA02609321
:103F5000BF027093C0028093C1029093C2029B0182
:103F6000AC010E942D39D10152966D937D938D93B2
:103F70009C935597077F0093A9020FC0F1016289B6
:103F80007389848995890E94CC396093BF027093AC
:103F9000C0028093C1029093C202F2E1FE9DC00173
:103FA000FF9D900D11249C01225B3D4F7901D901A9
:103FB00051961C928091700181FF1AC0F101818994
:103FC00085FF16C022A533A544A555A560E070E085
:103FD00080E89FE30E94D5366093D3027093D402A9
:103FE0008093D5029093D602E1E0D7015196EC93ED
:103FF0001092BB021092BC021092BD021092BE023F
:10400000D1015A962D913D914D915C915D972D83F3
:104010003E834F83588760E070E080E09FE30E941A
:10402000D5364B015C01F101468C578C60A071A024
:1040300011FF4BC0F2E0F093BA02D1015296CD903D
:10404000DD90ED90FC905597A70196010E942D39C7
:104050009B01AC01C301B2010E94D5354B015C014B
:1040600020E030E0A9010E94CB3687FF1DC02D81E2
:104070003E814F815885CA01B9010E94D635A301FE
:1040800092010E942D399B01AC01C701B6010E942B
:10409000D5350E94CC396093C7027093C8028093D3
:1040A000C9029093CA02A8C18092BB029092BC023E
:1040B000A092BD02B092BE021092C7021092C80236
:1040C0001092C9021092CA0297C11092BA0240928D
:1040D000CB025092CC026092CD027092CE0212FFBF
:1040E0000CC01092C7021092C8021092C90210921E
:1040F000CA02C12CD12C760124C0E091DA02EF5F14
:10410000E03109F4E0E08091FB058E1759F0B2E34D
:10411000BE9FF0011124E552FD4FC288D388E48888
:10412000F58803C0C12CD12C7601C701B6010E94CD
:10413000CC396093C7027093C8028093C9029093F0
:10414000CA02C1010E94381C698B7A8B8B8B9C8BB5
:104150009B01AC010E942D3969877A878B879C87E8
:10416000D10152962D913D914D915C9155972983A6
:104170003A834B835C830E94CB3687FF6CC02985D2
:104180003A854B855C8569817A818B819C810E940F
:10419000D535A50194010E942D399B01AC01C301C5
:1041A000B2010E94D5356093CB027093CC0280930C
:1041B000CD029093CE0220E030E0A9010E94CB36E0
:1041C00018163CF1B2E0B093BA022D813E814F81C6
:1041D0005885CA01B9010E94D635A30192010E94F7
:1041E0002D399B01AC0169817A818B819C810E9470
:1041F000D5350E94CC396093C7027093C802809372
:10420000C9029093CA028091A90288608093A90292
:10421000F3C0A701960169857A858B859C850E94EC
:10422000D535A50194010E942D396093CF0270937A
:10423000D0028093D1029093D20229893A894B8986
:104240005C892093C3023093C4024093C50250930B
:10425000C60233E0B6C0A701960169817A818B81DD
:104260009C810E94D535A50194010E942D39A3019E
:1042700092010E94D63520E030E040E05FE30E94EA
:104280002D396D877E878F87988B20E030E0A901DC
:104290000E94ED3818160CF097C02D853E854F858D
:1042A0005889C301B2010E94ED3818160CF088C07D
:1042B000A701960169857A858B859C850E94D535F5
:1042C000A50194010E942D399B01AC016093CF029E
:1042D0007093D0028093D1029093D2026D857E8537
:1042E0008F8598890E94ED381816CCF589899A89AE
:1042F000AB89BC898093C3029093C402A093C5028A
:10430000B093C60229813A814B815C8169857A85A7
:104310008B859C850E94CB36811104C091E09093DF
:10432000BA026AC029813A814B815C8169857A85AC
:104330008B859C850E94D535A50194010E942D395D
:104340009B01AC01C301B2010E94D5356093CB0241
:104350007093CC028093CD029093CE024DC02D85F8
:104360003E854F8558892093CB023093CC024093F1
:10437000CD025093CE022093CF023093D0024093CF
:10438000D1025093D2022D813E814F815885CA01BE
:10439000B9010E94D6352D853E854F8558890E94EA
:1043A0002D39A70196010E94D6350E94CC39609321
:1043B000C3027093C4028093C5029093C6021CC0CE
:1043C00032E03093BA0218C01092CB021092CC02A5
:1043D0001092CD021092CE028091C7029091C80235
:1043E000A091C902B091CA028093C3029093C40203
:1043F000A093C502B093C602186010931E0180916D
:104400004D02482F50E05E834D8387E0849FF0018A
:10441000859FF00D1124ED5DFD4F8091A8028483EE
:10442000A091FF05B0910006BFAFAEAF5E96BC9104
:10443000BEA3EEADFFADF78DFFA3AEADBFAD9096C1
:10444000BC91B8A7EEADFFADF1A1F9A72091B602DE
:104450003091B7024091B8025091B9026EA17FA18C
:104460008B2F9F2F0E94D5356AAB7BAB8CAB9DAB5E
:1044700020E030E0A9010E94CB3687FF04C01AAAD1
:104480001BAA1CAA1DAA2091CB0229873091CC021D
:104490003D874091CD02498B5091CE025D8B80913A
:1044A000C3028A8F9091C4029B8FA091C502AC8FEA
:1044B000B091C602BD8F6090BF027090C002409064
:1044C000C1025090C202E091CF02EAA7F091D0025F
:1044D000FBA72091D1022CA73091D2023DA7409199
:1044E000BA0249835091BB025EA78091BC028FA79C
:1044F0009091BD0298ABA091BE02A9ABB091C7024A
:10450000BFABE091C802E8AFF091C902F9AF2091CA
:10451000CA022AAF2AA53BA54CA55DA569857D8564
:1045200089899D890E94CB36811103C032E03EAB60
:1045300002C041E04EAB2EA03FA008A519A58EE316
:10454000C82E83ECD82E8EE2E82E89E3F82E1E8A40
:104550001F8A188E198ECE8EDF8EE8A2F9A299815D
:10456000913009F4D4C008F472C0AEADBFAD5A9614
:104570002D913D914D915C915D97933009F0F9C07B
:10458000C701B6010E942D394B015C0120E030E0EB
:1045900040E05FE30E942D399B01AC01B301C201F1
:1045A0000E94D535A70196010E942D396AA37BA3ED
:1045B0008CA39DA39B01AC01B101C8010E94D5351C
:1045C0001B018C0129853D8549895D890E94CB3677
:1045D00087FD0BC020E030E0A9016AA17BA18CA17E
:1045E0009DA10E94CB3618165CF129853D8549892D
:1045F0005D896EA17FA188A599A50E94D5359B01F3
:10460000AC010E94D6356B017C019301A2016A8D39
:104610007B8D8C8D9D8D0E94D6359B01AC01C70191
:10462000B6010E94D5366B017C016A8C7B8C4C8C68
:104630005D8C29843D8409891D89B1E0B983FFC05F
:10464000A5019401B301C2010E94D5355DC0EEAD54
:10465000FFAD228D338D448D558DC701B6010E946B
:104660002D394B015C0120E030E040E05FE30E9427
:104670002D399301A2010E94D635A70196010E940F
:104680002D399B01AC01B101C8010E94D5351B0138
:104690008C019B01AC0169857D8589899D890E947A
:1046A000ED3818165CF529853D8549895D896EA12F
:1046B0007FA188A599A50E94D5359B01AC010E94D8
:1046C000D6356B017C019301A2016A8D7B8D8C8DA7
:1046D0009D8D0E94D6359B01AC01C701B6010E9499
:1046E000D5366B017C016A8C7B8C4C8C5D8CFEA971
:1046F000F98329843D8409891D89A1C0A5019401FC
:10470000B301C2010E94D6353B012C0198C02A8D0D
:104710003B8D4C8D5D8DC701B6010E942D399B01EB
:10472000AC01B101C8010E94D5355B014C019B0170
:10473000AC016AA57BA58CA59DA50E94ED38181635
:104740000CF07BC02AA53BA54CA55DA5B101C80115
:104750000E94D5352A8D3B8D4C8D5D8D0E94D536BE
:104760006B017C012AA43BA40CA51DA522E0298392
:1047700066C0C701B6010E942D394B015C0193014F
:10478000A2010E94CB3687FF31C020E030E040E03C
:104790005FE3C501B4010E942D399B01AC01B30157
:1047A000C2010E94D535A70196010E942D399B01B7
:1047B000AC01B101C8010E94D5356AA37BAF8CAFB3
:1047C0009DAF2EA53FA548A959A90E94ED381816FE
:1047D0006CF4A5019401B301C2010E94D5353B01DF
:1047E0002C012AA03BAC0CAD1DAD29C02EA53FA5C8
:1047F00048A959A9B101C8010E94D5359B01AC0156
:104800000E94D6356B017C019301A2016FA978AD9E
:1048100089AD9AAD0E94D6359B01AC01C701B601A6
:104820000E94D5366B017C016FA878AC49AC5AACBC
:104830002EA43FA408A919A902C015018401A7014B
:1048400096016E897F89888D998D0E94D6356E8BF1
:104850007F8B888F998F2E8D3F8D48A159A10E9403
:10486000CB3687FF09C02E893F89488D598D6E8DC3
:104870007F8D88A199A11CC02AA93BA94CA95DA93B
:10488000B101C8010E94ED38181624F52EE333EC6F
:104890004EE259E36E8D7F8D88A199A10E94D63595
:1048A0006E8F7F8F88A399A32E893F89488D598D5C
:1048B0000E94D5356B017C019101A8016EA57FA5F1
:1048C00088A999A90E94CB3687FD49CEB981B093BA
:1048D000BA0203C0E981E093BA02C301D201809316
:1048E000BF029093C002A093C102B093C202E091B4
:1048F000FD05F091FE059189911104C080911E0182
:1049000083FF3FC0AEADBFAD51968C915197807380
:1049100049F19E96CD90DD90ED90FC90D197992332
:10492000D1F02091D3023091D4024091D502509120
:10493000D6026091BF027091C0028091C102909135
:10494000C2020E942D399B01AC01C701B6010E9431
:104950002D396B017C01C701B6010E943232809370
:10496000D7020AC010922701109228011092290143
:1049700010922A011092D70280911E01877F8093A6
:104980001E0147E02D813E81429FF001439FF00DC3
:104990001124ED5DFD4FFA87E9878091D702868368
:1049A0002091B2023091B3024091B4025091B5020D
:1049B000B101C8010E942D392B013C010E94B4367F
:1049C0006B017C016091AE027091AF028091B002E8
:1049D0009091B1020E94B4364B015C01A70196018F
:1049E0000E94D5350E944E3769837A838B839C83DE
:1049F000E981FA81A985BA85ED93FC93EF2B41F407
:104A000080911E0181FF04C0816080931E010AC154
:104A10002091AA023091AB024091AC025091AD02BC
:104A20006E897F89888D998D0E94D63569877A87AE
:104A30008B879C87A3019201C501B4010E94D535E3
:104A40009B01AC0169857A858B859C850E94D53652
:104A50004B015C0120EC31EE44E65EE40E942D390E
:104A60000E94B4360E944E37603D37E073078105DF
:104A7000910560F4A7E04D815E81A49FF001A59FA0
:104A8000F00D1124ED5DFD4F158253C0603ABFE07B
:104A90007B078105910560F447E02D813E81429FAF
:104AA000F001439FF00D1124ED5DFD4F51E011C069
:104AB0006034AFE17A078105910568F447E02D8104
:104AC0003E81429FF001439FF00D1124ED5DFD4FAB
:104AD00052E055830CC027E0AD81BE812A9FF001D2
:104AE0002B9FF00D1124ED5DFD4F33E03583A7E0E2
:104AF0004D815E81A49FF001A59FF00D1124ED5D15
:104B0000FD4F2581022E04C0969587957795679570
:104B10000A94D2F749815A8102C0440F551F2A9541
:104B2000E2F7518340836115710551E085079105D6
:104B300068F427E0AD81BE812A9FF0012B9FF00D24
:104B40001124ED5DFD4F7383628304C04FEF5FEF6F
:104B5000538342838091FC0580934D028F5F8630A2
:104B600019F08093FC0502C01092FC05E091FF054E
:104B7000F0910006C101D801868F978FA0A3B1A341
:104B8000C092AE02D092AF02E092B002F092B102B7
:104B9000A3019201C701B6010E94D535A501940178
:104BA0000E942D396093AA027093AB028093AC02ED
:104BB0009093AD022091BB023091BC024091BD02A6
:104BC0005091BE02B101C8010E94CB368111F4C8D8
:104BD00020E030E0A901B101C8010E94ED389091B8
:104BE0001E01181614F092FF04C0916090931E01EC
:104BF00019C0109200061092FF059091DA02809180
:104C0000FB05891709F4D8C881E0890F803109F4C0
:104C100080E02091D802921302C08093D802809342
:104C2000DA02CAC8EF960FB6F894DEBF0FBECDBF4A
:104C3000DF91CF911F910F91FF90EF90DF90CF9078
:104C4000BF90AF909F908F907F906F905F904F90AC
:104C50003F902F900895CF93DF93C091FF05D0919F
:104C600000062097C9F08091A90281608093A90273
:104C70006091BF027091C0028091C1029091C20206
:104C80009B01AC010E942D396A8B7B8B8C8B9D8B99
:104C9000109200061092FF05DF91CF9108952F9298
:104CA0003F924F925F926F927F928F929F92AF92BC
:104CB000BF92CF92DF92EF92FF920F931F93CF9309
:104CC000DF933090FB05311002C0D0E101C0D32D3D
:104CD000D150C091D802CD1709F416C1ED2EF12C98
:104CE00022E3D29F8001112405521D4FF801A688AE
:104CF000B788C08CD18C628D738D848D958D9B010E
:104D0000AC010E94D635F801268D378D40A151A106
:104D10000E942D394B018C019B01AC01B501C601EC
:104D20000E94CB3687FD02C05401680182E38E9D4C
:104D3000F0018F9DF00D1124E552FD4FC501D60104
:104D4000828B938BA48BB58BD11101C0D0E1D15054
:104D5000CD1307C08091DA02C81368C00E942B26C9
:104D600065C022E32E9DC0012F9D900D11249C0152
:104D700025523D4F790192E3292EAD2EB12C2A9C6C
:104D8000C0012B9C900D1124FC01E552FD4F6F01D9
:104D9000D11101C0D0E1D1508091DA028D1302C04F
:104DA0000E942B262A9C80012B9C100D1124055259
:104DB0001D4FF80186889788A08CB18CA5019401BD
:104DC00062897389848995890E94CB36882359F139
:104DD000F801628D738D848D958D9B01AC010E94CD
:104DE000D635F801268D378D40A151A10E942D396D
:104DF000F70122893389448955890E94D6352B01D0
:104E00003C019B01AC01C501B4010E94ED38F801E1
:104E100018162CF4428A538A648A758A04C0828ADE
:104E2000938AA48AB58A7601CD13A7CFF2E3CF9FE8
:104E30008001112405521D4FCF5FC03109F4C0E03D
:104E4000D091D80282E3282EC31509F45BC0CC2E82
:104E5000D12C2C9CC0012D9C900D11249C0125521D
:104E60003D4F7901F8014288538864887588F901BB
:104E700082889388A488B588A5019401C301B201F2
:104E80000E94CB3687FF24C0F801628D738D848D1C
:104E9000958D9B01AC010E94D635F801268D378D8A
:104EA00040A151A10E942D39A30192010E94D63543
:104EB0002B013C019B01AC01C501B4010E94ED38FE
:104EC000181634F4F701428A538A648A758ADC2FF3
:104ED0002C9CF0012D9CF00D1124E552FD4F2689EC
:104EE0003789408D518D62897389848995890E94A3
:104EF000CB36811101C0DC2FCF5FC03109F4C0E097
:104F00008701A2CFD093D802DF91CF911F910F914B
:104F1000FF90EF90DF90CF90BF90AF909F908F90D9
:104F20007F906F905F904F903F902F9008952F92B9
:104F30003F924F925F926F927F928F929F92AF9229
:104F4000BF92CF92DF92EF92FF920F931F93CF9376
:104F5000DF93CDB7DEB7C454D1090FB6F894DEBFE6
:104F60000FBECDBF3B010091FB05202E312C22E36B
:104F7000229DA001239D500D1124BA0165527D4F41
:104F80007AAF69AFFB0111922A95E9F7F301208509
:104F9000FB01218BF3014481558166817781E9AD65
:104FA000FAAD46A757A760AB71AB21FF40C02CE01C
:104FB000E1E0F1E0DE01599601900D922A95E1F7CA
:104FC0008BAB9CAB2BE231E03EAB2DABBE01635F04
:104FD0007F4F23967FAF6EAF2397CE0149962196E0
:104FE0009FAF8EAF2197E2E30E9FC00111249C0179
:104FF00025523D4F3EAF2DAF685E7F4F7CAF6BAF0C
:1050000078AF6FAB10E082E3829D9001839D300DFD
:105010001124C90185529D4FFC013C962596FFAF96
:10502000EEAF25972C01F0E14F0E511C3CC02CE057
:10503000E1E0F6E0BFCFEDADFEAD219331934193BA
:105040005193FEAFEDAF2596EEADFFAD2597C08035
:10505000D180E280F380C216D306E406F50610F490
:1050600069017A012596EEADFFAD2597C082D18208
:10507000E282F3820E947F37A50194010E94D53617
:10508000EFA9F8AD6193719381939193F8AFEFAB72
:1050900020E030E0A9010E94CB3687FD42C01F5FAF
:1050A000133009F44CC0EBA9FCA961917191819175
:1050B0009191FCABEBABEDA9FEA981909190A190F1
:1050C000B190FEABEDABA50194010E942D390E9479
:1050D000FA382396EEADFFAD2397619371938193D8
:1050E00091932396FFAFEEAF23972196EEADFFADE0
:1050F0002197C190D190E190F1902196FFAFEEAF52
:1051000021976C197D098E099F099B01AC0197FFBE
:1051100092CF22273327A901261B370B480B590BA7
:105120008ACF112321F0113021F080E803C080E202
:1051300001C080E4F2019081892B8083B0CFCD281B
:10514000CE28CF2809F496C1CE0185960E94303131
:105150004B015C0122E3229DC001239D900D11248F
:105160009C0125523D4F7901F901868E978EA0A2B0
:10517000B1A2BE016B5D7F4F83E491E00E94DA3003
:10518000F701628F738F848F958FBE016B5D7F4FA8
:1051900087E391E00E94DA30F70166A377A380A746
:1051A00091A7118910FD12C0F30120813181428144
:1051B000538113FD06C0F70122A733A744A755A7C3
:1051C00009C0C501B4010E942D39F70162A773A778
:1051D00084A795A78091DA02081711F011FF0DC07E
:1051E00082E3829DF001839DF00D1124E552FD4F75
:1051F000128A138A148A158A54C02DE036E03CAB1B
:105200002BAB8E010F5F1F4FBE016F5C7F4F7AABE0
:1052100069ABC12CD12C76010DAB1FABEBA9FCA95E
:1052200081909190A190B190FCABEBABEBADFCAD5C
:105230004190519061907190FCAFEBAFA30192014E
:10524000C501B4010E942D399B01AC01C701B60113
:105250000E94D5356B017C01A5019401C301B20107
:105260000E94D535F80161937193819391938F01D9
:1052700029A93AA96BAD7CAD2617370779F62FEE31
:105280003FEF4FE75FE3C701B6010E94ED38181604
:105290006CF482E3829DF001839DF00D1124E552B0
:1052A000FD4F12A213A214A215A271C02FEE3FEF60
:1052B0004FE75FEBC701B6010E94CB3687FF11C0F5
:1052C00082E3829DF001839DF00D1124E552FD4F94
:1052D00089E996E7A6E9BEE782A393A3A4A3B5A3B1
:1052E00056C08DA99FA90E9430316DA97FA983E482
:1052F00091E00E94DA304B015C01A701960160E069
:1053000070E080E89FE30E94D53520E030E040E087
:105310005FE30E942D390E94CC396B017C01209102
:105320006001309161014091620150916301C501BA
:10533000B4010E942D39A70196010E942D394B011D
:105340005C01A701960160E070E080E89FE30E94A5
:10535000D5359B01AC01C501B4010E94D5366B0166
:105360007C0120E030E0A9010E94CB3687FF03C01A
:10537000C12CD12C760182E3829DF001839DF00D3A
:105380001124E552FD4FC2A2D3A2E4A2F5A282E30A
:10539000829D8001839D100D112405521D4FF8013F
:1053A000818981FD69C089AD9AAD0E94381C6B016D
:1053B0007C018090190690901A06A0901B06B09070
:1053C0001C06A50194010E94ED3818162CF4A501C5
:1053D0009401C501B40104C0A7019601C701B6013B
:1053E0000E942D39F801668B778B808F918F82E335
:1053F000829D8001839D100D112405521D4FF801DF
:1054000082A093A0A4A0B5A0A50194016689778984
:10541000808D918D0E94ED3818162CF4F801868A43
:10542000978AA08EB18EC0921906D0921A06E09289
:105430001B06F0921C068CE0FE01B596ADE0B6E0CE
:1054400001900D928A95E1F78CE0FE013D96A1E076
:10545000B6E001900D928A95E1F78091D902809390
:10546000FB058F5F803109F480E08093D9020E94B0
:105470004F2602C080E001C081E0CC5BDF4F0FB659
:10548000F894DEBF0FBECDBFDF91CF911F910F917A
:10549000FF90EF90DF90CF90BF90AF909F908F9054
:1054A0007F906F905F904F903F902F900895CF9393
:1054B000DF930E944F1580E3E8EAF2E0DF011D92DE
:1054C0008A95E9F7CFEFD1E083E2FE0111928A9548
:1054D000E9F7109200061092FF0510922202109236
:1054E0004D0281E08093FC051092FE010E941E1582
:1054F0008091FD018F878BB1837E9091FC01892B78
:105500008BB98BB18F719091FD01892B8BB9DF9194
:10551000CF910895CF93DF93C1E1D7E0899188239C
:1055200019F00E940932FACFDF91CF910895CF93FD
:10553000DF9321E5829FC0011124EC01DD5F40E58E
:1055400050E0BE0181E197E00E94591E892B69F469
:10555000109211070E94F93340E550E061E177E0D5
:10556000CE010E94CC1C80E001C081E0DF91CF9190
:1055700008959FB7F89420912006822B80932006EF
:105580009FBF08959FB7F89420911F06822B8093A8
:105590001F069FBF08959FB7F89480931E069FBF74
:1055A00008952FB7F89490911D06809589238093D4
:1055B0001D062FBF08959FB7F89420911D06822BDA
:1055C00080931D069FBF08958F929F92AF92BF92C6
:1055D000EF92FF920F931F93CF93DF93EC010FE4B1
:1055E00011E07C018CE0E80EF11C89909990A99063
:1055F000B99020E030E0A901C501B4010E94CB368A
:1056000087FD14C0F80181919191A191B1918F0111
:105610009C01AD015058C501B4010E94ED38181627
:105620002CF0CE15DF0509F780E001C081E0DF91A5
:10563000CF911F910F91FF90EF90BF90AF909F90EF
:105640008F9008958F929F92AF92BF92CF92DF92E8
:10565000EF92FF920F931F93CF93DF93EB012BE217
:10566000E22E21E0F22E8C016B018CE0C80ED11CE1
:105670006991799189919991F70181909190A19087
:10568000B1907F010E947F37A50194010E94D53619
:10569000F80161937193819391938F01CC15DD058E
:1056A00039F7DF91CF911F910F91FF90EF90DF902D
:1056B000CF90BF90AF909F908F9008950E94F93344
:1056C00010922601089596B1892F877049F0892F8D
:1056D0008095817091FF826092FD03C0846008957F
:1056E00080E008951F920F920FB60F9211242F930E
:1056F0003F934F935F936F937F938F939F93AF935A
:10570000BF93EF93FF930E94632B882391F080FF58
:1057100003C00E9461340DC082FF04C080911D0649
:10572000826005C081FF05C080911D06886080935E
:105730001D06FF91EF91BF91AF919F918F917F9146
:105740006F915F914F913F912F910F900FBE0F90EE
:105750001F901895109200019091700197FD03C061
:1057600090E290930001882331F09091000180E253
:1057700089278093000108958F929F92AF92BF92E4
:10578000CF92DF92EF92FF920F931F93CF93DF930D
:10579000CDB7DEB72D970FB6F894DEBF0FBECDBFE5
:1057A0006B017C01042F20E030E0A9010E94CB3680
:1057B00087FF07C08DE20E940932F7FAF094F7F8EC
:1057C000F094102F123060F020E030E048EC52E40A
:1057D000C701B6010E942D396B017C011250F2CF36
:1057E00000FF0AC020E030E040E251E4C701B6010A
:1057F0000E942D396B017C0120E030E040E05FE346
:10580000C701B6010E94D6350E94473710E03AE042
:10581000832E912CA12CB12C611571058105910568
:1058200091F0EE24E394F12CEC0EFD1EE10EF11C40
:10583000A50194010E94563A605DF7016083B901A9
:10584000CA011F5FE9CF80E3101748F4E1E0F0E000
:10585000EC0FFD1FE10FF11D80831F5FF5CF1013CB
:1058600013C0FE01E10FF11D80E381831F5F0CC0B7
:10587000101303C08EE20E940932FE01E10FF11DF8
:1058800080810E94093211501111F2CF2D960FB66E
:10589000F894DEBF0FBECDBFDF91CF911F910F9166
:1058A000FF90EF90DF90CF90BF90AF909F908F9040
:1058B00008952091700120FF08C02BE832E441E2F6
:1058C0005DE30E942D3941E001C040E00C94BC2B07
:1058D0002091700120FF08C02BE832E441E25DE333
:1058E0000E942D3944E001C043E00C94BC2B0F937F
:1058F0001F93CF938C01C0E0F80161917191819168
:1059000091918F010E94682CC23019F08CE20E94A4
:105910000932CF5FC33081F7CF911F910F91089566
:10592000CF93DF93843630F06AE00E94363AC0E3CA
:10593000C90F03C0C0E08A3030F06AE00E94363AF6
:10594000D0E3D90F01C0D0E0805D0E940932DD2391
:1059500019F08D2F0E940932CC2329F08C2FDF9172
:10596000CF910C940932DF91CF910895CF93DF93BB
:10597000FC018491EF012196882321F00E940932D5
:10598000FE01F7CFDF91CF9108958CE093E00C9466
:10599000B62CCF93C82F85E193E00E94B62C8C2FB4
:1059A0000E94902CCF910C94C52C811104C08CE1E5
:1059B00093E00C94B62C0C94C92CCF93DF93C0E0E9
:1059C0008C2F0E94972A81110EC0109211078EE32E
:1059D0000E9409320E948A2A8AE30E94093287E0E3
:1059E0000E94C92C12C080911107882371F00E9477
:1059F000A501D82F8EE30E9409320E948A2A8AE3E9
:105A00000E9409328D2F0E94D52CCF5FC230C1F683
:105A1000DF91CF910895CF92DF92EF92FF92CF93D3
:105A2000DF93D82F6A017B01C22F84E20E940932E2
:105A30008D2F0E94902C8DE30E9409324C2FC701BC
:105A4000B6010E94BC2BDF91CF91FF90EF90DF90C9
:105A5000CF900C94C52CCF93DF93D82FC62F84E220
:105A60000E9409328D2F0E94902C8DE30E940932F2
:105A70008C2F0E94902CDF91CF910C94C52CEF922B
:105A8000FF920F931F93CF93DF9360915B0170E0C0
:105A900080E00E942B2D60915E0170E081E00E9409
:105AA0002B2D60915C0170E082E00E942B2D6091B3
:105AB0005D0170E083E00E942B2D6091700162FB1C
:105AC000662760F970E084E00E942B2D60917001E0
:105AD00066FB662760F970E085E00E942B2D8091BF
:105AE0007001082E000C990B692F661F6627661F30
:105AF00070E086E00E942B2D60915F0170E08AE0EB
:105B00000E942B2D409160015091610160916201D2
:105B10007091630123E08BE00E940B2D40916401A2
:105B200050916501609166017091670123E08CE0FE
:105B30000E940B2D60917001617070E08DE00E94F9
:105B40002B2D6091700165FB662760F970E084E1A0
:105B50000E942B2D6091700163FB662760F970E055
:105B600085E10E942B2D609170016295617070E05B
:105B700086E10E942B2D6091710170E087E10E9407
:105B80002B2D4091720150917301609174017091BD
:105B9000750123E088E10E940B2D40917601509120
:105BA0007701609178017091790123E089E10E9489
:105BB0000B2D60917A0170917B018AE10E942B2D5F
:105BC00040917C0150917D0160917E0170917F0137
:105BD00023E08BE10E940B2D4091680150916901F7
:105BE00060916A0170916B0120E08EE10E940B2DA3
:105BF00040916C0150916D0160916E0170916F0147
:105C000020E08FE10E940B2D60917001669561701C
:105C100070E080E20E942B2DD4E6F12C0BE211E023
:105C200083E0E82EED0ECD2F82E0F81691F0E3E050
:105C3000FE16E9F0F1E0FF1631F0F80140815181E4
:105C4000628173811AC0F801448555856685778520
:105C500014C020E030E041E655E4F801608D718D1C
:105C6000828D938D0E94D536AB01BC0106C0F80130
:105C700044A155A166A177A1705823E08C2F0E9402
:105C80000B2D0C5F1F4FCF5FEC12CECFD65FF3947E
:105C9000DC3821F6DF91CF911F910F91FF90EF90AB
:105CA00008958DE50E9409320C94C52CCF93DF93A3
:105CB000CDB7DEB72C970FB6F894DEBF0FBECDBFC1
:105CC0008FE093E00E94B62C6DE071E0CE0101966A
:105CD0000E94222BCE0101960E94772C8AE30E941B
:105CE000093280911F010E94902C0E94512E2C9607
:105CF0000FB6F894DEBF0FBECDBFDF91CF910895F0
:105D00001F920F920FB60F9211242F933F934F9330
:105D10005F936F937F938F939F93AF93BF93EF9313
:105D2000FF9380911A01813049F080911E06811104
:105D300005C00E94613481E00E94CB2AFF91EF915F
:105D4000BF91AF919F918F917F916F915F914F9193
:105D50003F912F910F900FBE0F901F90189593B108
:105D600096718091700186FD02C086E19827992383
:105D700049F091FB882780F992FD8260907119F0BB
:105D80008460089580E008952F923F924F925F9231
:105D90006F927F928F929F92AF92BF92CF92DF923B
:105DA000EF92FF920F931F93CF93DF93CDB7DEB7A0
:105DB000A1970FB6F894DEBF0FBECDBF90911B0127
:105DC0009111BDC18D8FFE013D9689E0DF011D92CD
:105DD0008A95E9F786E08D8BEBE2F1E0FA8FE98FA7
:105DE0005F019E012A5E3F4F490100E010E0C12C97
:105DF000D12C76019D8D892F90E09C8F8B8F802FE9
:105E0000002321F0013021F090E103C094E001C0B3
:105E100098E0D4019D934D01EB8DFC8D02C0F5956A
:105E2000E7958A95E2F7E0FF1BC020E030E040EC08
:105E30005FEBD50194966D917D918D919C91979793
:105E40000E942D39362E472E582E692EA701960115
:105E50000E94CB3687FD04C0C32CD42CE52CF62C35
:105E60000F5F1F4FB4E0AB0EB11C0330110539F6C4
:105E70002090760130907701409078015090790120
:105E800094E0A92EBB24B39461E071E0CE010196A9
:105E90000E94222B80917101E82FF0E0FF8FEE8F9E
:105EA000FE01319681E0682E81E0782E79A268A209
:105EB000CE0146964C0180E090E000E010E0B70192
:105EC000A60170582B8D3C8D082E02C03595279564
:105ED0000A94E2F720FF23C00F5FA8A1B9A11D9289
:105EE0001D921D921C9213972E8D3F8D082E02C07D
:105EF000359527950A94E2F720FF03C0BB2019F0DF
:105F000007C0BB2029F0C082D182E282F38204C0A4
:105F10004083518362837383D4012C91122B0196A9
:105F2000BFEF8B1A9B0A349628A139A12C5F3F4FF3
:105F300039A328A38330910529F6602F70E080E013
:105F400090E00E947D370E94CC399B01AC011093F8
:105F50002001C201B1010E942D396D877E878F8794
:105F6000988BBE01635F7F4FCE0101960E949727F9
:105F700034E030931E010E94BE1E0E94CD17BB204C
:105F8000E9F00E94AF2EFE01769620E030E090E02E
:105F90006191462F412359F0AC01022E02C0559564
:105FA00047950A94E2F740FF02C0609516232F5FE1
:105FB0003F4F2330310561F7109320010E94BE1E30
:105FC00080911D06847339F110911D0614FF03C0E2
:105FD00086E00E94CB2A15FF03C087E00E94CB2AEF
:105FE000B11007C00E94AF2E9D8D892339F088E043
:105FF00003C012FF03C089E00E94CB2A80911E06D5
:10600000882329F00E9461340E94ED3298C084E018
:106010000E94D12A04C0812F8C7109F0B0CF0E9458
:10602000572A00917A0110917B010115110549F061
:10603000AFE9BFE01197F1F700C00000015011096E
:10604000F4CFB1E0BB26C9F020E030E040EA50E4F4
:1060500060917C0170917D0180917E0190917F0122
:106060000E942D396B017C012090720130907301E8
:10607000409074015090750110C0C0907C01D09088
:106080007D01E0907E01F0907F01209076013090BC
:1060900077014090780150907901AA94A110F4CE34
:1060A000E0907101F12C80907C0190907D01A09096
:1060B0007E01B0907F018B8D9C8D002E02C0959546
:1060C00087950A94E2F780FF29C0C701002E02C01D
:1060D000959587950A94E2F780FD18C0E98DFA8DB1
:1060E00084A195A1A6A1B7A1BC01CD019058A5019D
:1060F00094010E94D535A98DBA8D2D913D914D9178
:106100005C910E942D390E94FA3803C060E070E073
:10611000CB01F30160837183828393830F5F1F4FF1
:10612000F4E06F0E711C298D3A8D2C5F3F4F3A8F32
:10613000298F0330110509F0BECF10921E01A196E0
:106140000FB6F894DEBF0FBECDBFDF91CF911F9188
:106150000F91FF90EF90DF90CF90BF90AF909F9006
:106160008F907F906F905F904F903F902F90089509
:10617000EBE6F0E08081897E8083E8E6F0E08081D4
:106180008E7F8083089584B1897E84B985B18661CC
:1061900085B98091700183FF0BC080916B0086618F
:1061A00080936B00809168008160809368000895FF
:1061B0000C94B8306F927F928F929F92AF92BF9261
:1061C000CF92DF92EF92FF920F931F93CF93DF93C3
:1061D000EB018C015B018CE0A80EB11C89E9682EF3
:1061E00096E7792E26E9822E3EE7932EC990D99024
:1061F000E990F99020E030E0A901C701B6010E94C2
:10620000CB368823B9F0A7019601F801608171812E
:10621000828193810E94D5366B017C01E894F7F866
:106220009301A401C701B6010E94ED38181614F0BD
:10623000360147010C5F1F4FCA15DB05B9F6B301E4
:10624000C401DF91CF911F910F91FF90EF90DF90EC
:10625000CF90BF90AF909F908F907F906F90089558
:106260004F925F926F927F92AF92BF92CF92DF92E6
:10627000EF92FF920F931F93CF93DF93EC015C019A
:106280008CE0A80EB11C8E01C12CD12C7601F80136
:1062900041905190619071908F0120E030E0A90110
:1062A000C301B2010E94CB36882371F0A301920191
:1062B000C301B2010E942D399B01AC01C701B60197
:1062C0000E94D6356B017C010A151B0501F7C70139
:1062D000B6010E94CC396B017C019B01AC0160E0EE
:1062E00070E080E89FE30E94D5362B013C01A301BA
:1062F0009201688179818A819B810E942D396993FD
:10630000799389939993AC16BD0689F7C701B601B5
:10631000DF91CF911F910F91FF90EF90DF90CF9081
:10632000BF90AF907F906F905F904F9008951F93B4
:10633000CF93DF93142F20E030E040EA51E40E9435
:106340002D390E94B4360E944E37EB012097D1F0D0
:1063500080911B01811116C0111103C00E94ED3202
:1063600006C00E94E51780911C0181FD0BC02FEF34
:1063700080E792E0215080409040E1F700C00000AB
:106380002197E4CFDF91CF911F910895E1E0F1E0F3
:10639000A1E0B6E041915191619171914D935D936E
:1063A0006D937D9381E0ED30F807A1F708950E9489
:1063B000AB1C892B19F082E00C94DB2A08951F9204
:1063C0000F920FB60F9211248F939F93EF93FF9329
:1063D00080911007E82FF0E0E955F94F90819093F4
:1063E000C6008F5F893609F480E080931007909192
:1063F000A606891305C08091C1008F7D8093C100DE
:10640000FF91EF919F918F910F900FBE0F901F9072
:106410001895E091A60691E09E0F993631F490E030
:1064200004C020911D0624FD0FC0209110072917DC
:10643000C1F3F0E0E955F94F80839093A60680916F
:10644000C10080628093C100089590911B01911159
:1064500008C0811102C0439802C086FD439A109281
:10646000250108954F925F926F927F928F929F9233
:10647000AF92BF92CF92DF92EF92FF926B017C01BD
:1064800080906C0190906D01A0906E01B0906F01B2
:10649000409068015090690160906A0170906B01B2
:1064A000A3019201C501B4010E94ED3887FF08C025
:1064B000A7019601C301B2010E94CB36181654F011
:1064C00040922701509228016092290170922A017E
:1064D00086E23CC0A7019601C501B4010E94ED38D7
:1064E00087FD11C020E030E0A901C701B6010E947C
:1064F000CB368092270190922801A0922901B09278
:106500002A0187E023C0C0922701D0922801E0929F
:106510002901F0922A01A5019401C701B6010E9448
:10652000D5352091A2063091A3064091A406509142
:10653000A5060E942D390E94BA3720E030E040EED7
:1065400050E40E94D6350E944E37862FFF90EF9080
:10655000DF90CF90BF90AF909F908F907F906F9083
:106560005F904F9008958093B300811104C0809193
:10657000B0008F7703C08091B00080688093B00036
:10658000089590911B01911127C081110FC080E0E7
:1065900090E0A0EEB0E48093270190932801A093AF
:1065A0002901B0932A01BC01CD0110C0803111F442
:1065B0002D9801C02D9A9091700191FF05C08032F5
:1065C00019F440E050E0BA01CB01BA010E94323226
:1065D0000E94B332109225010895CF92DF92EF927C
:1065E000FF921F93CF93DF930E94E51780911C01C8
:1065F000882309F4F6C00E94AB1C009771F4C09187
:10660000890180918801C82BC0908B01D0908C01AA
:10661000E0908D01F0908E0106C0FC01C189C6A4F6
:10662000D7A4E0A8F1A88091700181FF03C080E2A7
:106630000E94B92ADC2FD07311E0C07480911C0134
:10664000882309F4CEC090911B019111CAC080FF2C
:10665000C5C090911A01292F207C09F474C082FDD5
:1066600012C01092240140E050E0BA0180E00E9484
:10667000C13280E00E94253280911C018D7F8460B0
:1066800080931C01ABC09038E1F481EF91E00E944F
:10669000B62C8AE591E00E94B62C0E94512E40E073
:1066A00050E0BA0180E00E94C13280E00E942532B1
:1066B0000E944F1580911B01811193C00E94E51724
:1066C000F9CF903419F48F7D80931C0180911C01C7
:1066D00083FF84C0909189019923C1F081FD16C088
:1066E0008091700181FF06C080911E0188608093B7
:1066F0001E010CC0B701A6018D2F0E94C13241E0DE
:1067000060E070E080E890E40E9497318091880119
:10671000882371F080911C0181FD0AC08C2F0E949A
:10672000253241E060E070E080E89FE30E9497310D
:1067300080911C0181FD52C0806180931C0182E028
:106740000E94DB2A4BC0809124018823C9F181FF7C
:106750000DC0809189018823B1F040E050E0BA017A
:1067600080E00E94C1321093240138C08C70B1F1D6
:106770008091890181110AC08091240183FF03C0A7
:1067800082E00E94DB2A1092240128C081EF91E070
:106790000E94B62C83E691E00E94B62C0E94512EF6
:1067A0008091700181FF06C080911E0188608093F6
:1067B0001E01E2CFB701A6018D2F0E94C132DCCFAE
:1067C00080911E0183FF0AC0B701A6018D2F0E9490
:1067D000C13280911E01877F80931E010E94E517C0
:1067E0002DCFDF91CF911F91FF90EF90DF90CF9051
:1067F00008950E94D7310E94ED3280911B018111D2
:1068000008C00E94AB1C892BB1F780911A01883017
:1068100091F30895CF92DF92EF92FF92CF939091F0
:106820001A01923079F06A017B01C82F0E94F93376
:10683000B701A6018C2FCF91FF90EF90DF90CF9002
:106840000C94C132CF91FF90EF90DF90CF900895DC
:10685000CF93DF93239AC0EBD0E083E0888387E077
:106860008093B100259A20916C0130916D01409187
:106870006E0150916F016091680170916901809182
:106880006A0190916B010E94D5359B01AC0160E0DB
:1068900070E088EF91E40E94D5366093A206709371
:1068A000A3068093A4069093A50688818F7788839A
:1068B000DF91CF91089561E071E088E991E00C9457
:1068C000222B80911D0684FD1FC080E10E94DB2ADF
:1068D0008091B0008F778093B000439890911A0117
:1068E000892F8C7221F480911E01867069F094309A
:1068F00031F480911E06811105C086E001C083E05D
:106900000E94CB2A0C944F1508951F920F920FB638
:106910000F9211242F933F934F935F936F937F9325
:106920008F939F93AF93BF93EF93FF93E091C60034
:10693000E13271F028F4E83179F40E94613456C0F4
:10694000EF3321F0EE3741F482E003C081E001C073
:1069500088E00E94DB2A4AC0E7FF37C08E2F90E014
:10696000FC01E458F109ED31F10508F03FC0E659AA
:10697000FF4F0C94783A80E2ECCF80911A0185FFAA
:1069800035C080E4E6CF81E00DC082E00BC084E03A
:1069900009C088E007C080E105C080E203C080E450
:1069A00001C080E80E94C22A21C081E00BC082E0C1
:1069B00009C084E007C088E005C080E103C080E230
:1069C00001C080E40E94B92A11C0A091FA0181E0BF
:1069D0008A0F813809F480E09091FB01891731F02A
:1069E000B0E0AF5DB94FEC938093FA01FF91EF9166
:1069F000BF91AF919F918F917F916F915F914F91D7
:106A00003F912F910F900FBE0F901F901895CF932D
:106A1000C82F0E94B830CC2311F08C2F01C083E026
:106A20000E94C42E0E94ED3280911B01811107C08B
:106A30000E945B340E94C631CF910C94C330CF9139
:106A400008958F929F92AF92BF92CF92DF92EF9272
:106A5000FF920F931F93CF93DF937C016B01DC01B7
:106A6000CC91D0E0FE01EF5EF84F80818D3229F4A9
:106A7000EF012296818101E009C08B3219F0CE5ED0
:106A8000D84F03C0EF012296818100E0912CF0E005
:106A900010E020E030E0A9015E01E0EDE80FEA300F
:106AA000D0F4FF5FF93098F491101150A5E0B0E0F8
:106AB0000E947E3ADC01CB01880F991FAA1FBB1FE1
:106AC0009C01AD012E0F311D411D511D0AC09110B9
:106AD00008C01F5F06C0EE3F41F4911006C0992424
:106AE00093942196D5018C91D7CFFF2309F44FC001
:106AF000CA01B9010E947D374B015C0120E030E002
:106B0000A9010E94CB36882349F11F3F64F42AE093
:106B100037ED43E25CE3C501B4010E942D394B011E
:106B20005C011E5FF2CF1F3F59F42DEC3CEC4CECA6
:106B30005DE3C501B4010E942D394B015C010EC01B
:106B4000112361F020E030E040E251E4C501B401DE
:106B50000E942D394B015C011150F2CF002351F0FE
:106B6000B7FAB094B7F8B094F60180829182A2820D
:106B7000B38206C0D6018D929D92AD92BC921397BE
:106B8000C151D740C150F701C08381E001C080E00E
:106B9000DF91CF911F910F91FF90EF90DF90CF90F9
:106BA000BF90AF909F908F9008955058BB27AA2711
:106BB0000E94ED350C9487380E944E3838F00E94C0
:106BC000553820F039F49F3F19F426F40C942438FA
:106BD0000EF4E095E7FB0C94F537E92F0E94AC38F2
:106BE00058F3BA17620773078407950720F079F402
:106BF000A6F50C94E6380EF4E0950B2EBA2FA02DD6
:106C00000B01B90190010C01CA01A0011124FF2759
:106C1000591B99F0593F50F4503E68F11A16F04054
:106C2000A22F232F342F4427585FF3CF4695379553
:106C30002795A795F0405395C9F77EF41F16BA0B18
:106C4000620B730B840BBAF09150A1F0FF0FBB1FC6
:106C5000661F771F881FC2F70EC0BA0F621F731F0F
:106C6000841F48F4879577956795B795F7959E3F6C
:106C700008F0B0CF9395880F08F09927EE0F9795FD
:106C8000879508950E944E3860F080E891E009F4FD
:106C90009EEF0E94553828F040E851E071F45EEF15
:106CA0000CC00C9424380C94E638E92FE0780E944C
:106CB000AC3840F3092E052AB1F3261737074807E9
:106CC000590738F00E2E07F8E02569F0E025E0645A
:106CD0000AC0EF6307F8009407FADB01B9019D01D0
:106CE000DC01CA01AD01EF930E94EC360E948738A7
:106CF0000E9485365F91552339F02BED3FE049E442
:106D000050FD49EC0C94D6350895DF93DD27B92F5B
:106D1000BF7740E85FE31616170648075B0718F4CD
:106D2000D92F0E94F2389F938F937F936F930E9485
:106D30000C3AEEE0F1E00E9427380E9487382F914C
:106D40003F914F915F910E944039DD2351F090585F
:106D5000A2EA2AED3FE049EC5FE3D0785D270E948C
:106D6000ED35DF910C9487380E94CE3890F09F3734
:106D700048F4911116F40C94E73860E070E080E874
:106D80009FE3089526F01B16611D711D811D0C9453
:106D9000FB370C9416380E94D13708F481E008952F
:106DA0000E945E38E3950C9498380E94E9360C9462
:106DB00087380E94553858F00E944E3840F029F428
:106DC0005F3F29F00C94F53751110C94E7380C947F
:106DD00024380E94AC3868F39923B1F3552391F31A
:106DE000951B550BBB27AA2762177307840738F03A
:106DF0009F5F5F4F220F331F441FAA1FA9F335D097
:106E00000E2E3AF0E0E832D091505040E695001C4A
:106E1000CAF72BD0FE2F29D0660F771F881FBB1F04
:106E2000261737074807AB07B0E809F0BB0B802DE2
:106E3000BF01FF2793585F4F3AF09E3F510578F00E
:106E40000C94F5370C94E7385F3FE4F3983ED4F3A5
:106E5000869577956795B795F7959F5FC9F7880FE2
:106E6000911D9695879597F90895E1E0660F771F34
:106E7000881FBB1F621773078407BA0720F0621BC5
:106E8000730B840BBA0BEE1F88F7E09508950E94F0
:106E90004E376894B1110C94E73808950E94B438C5
:106EA00088F09F5798F0B92F9927B751B0F0E1F0CB
:106EB000660F771F881F991F1AF0BA95C9F714C07B
:106EC000B13091F00E94E638B1E008950C94E638B4
:106ED000672F782F8827B85F39F0B93FCCF38695B4
:106EE00077956795B395D9F73EF490958095709511
:106EF00061957F4F8F4F9F4F0895E89409C097FB8E
:106F00003EF490958095709561957F4F8F4F9F4F80
:106F10009923A9F0F92F96E9BB279395F6958795C4
:106F200077956795B795F111F8CFFAF4BB0F11F487
:106F300060FF1BC06F5F7F4F8F4F9F4F16C088232E
:106F400011F096E911C0772321F09EE8872F762F64
:106F500005C0662371F096E8862F70E060E02AF0A5
:106F60009A95660F771F881FDAF7880F9695879591
:106F700097F908950E94CE3890F09F3748F4911108
:106F800016F00C94E73860E070E080E89FEB08951D
:106F900026F41B16611D711D811D0C94FB370C948A
:106FA0001638990F0008550FAA0BE0E8FEEF1616E9
:106FB0001706E807F907C0F012161306E407F507ED
:106FC00098F0621B730B840B950B39F40A2661F061
:106FD000232B242B252B21F408950A2609F4A14004
:106FE000A6958FEF811D811D089597F99F6780E811
:106FF00070E060E00895882371F4772321F09850C1
:10700000872B762F07C0662311F499270DC0905166
:10701000862B70E060E02AF09A95660F771F881F34
:10702000DAF7880F9695879597F908959F3F31F085
:10703000915020F4879577956795B795880F911DA6
:107040009695879597F908959FEF80EC0895DF93C3
:10705000CF931F930F93FF92EF92DF927B018C01EE
:10706000689406C0DA2EEF010E944039FE01E894D0
:10707000A5912591359145915591A6F3EF010E9477
:10708000ED35FE019701A801DA9469F7DF90EF90E2
:10709000FF900F911F91CF91DF91089500240A94E2
:1070A0001616170618060906089500240A941216E3
:1070B00013061406050608950C9424380E94B4386B
:1070C000D8F3E894E0E0BB279F57F0F02AED3FE0CB
:1070D00049EC06C0EE0FBB0F661F771F881F28F014
:1070E000B23A62077307840728F0B25A620B730B37
:1070F000840BE3959A9572F7803830F49A95BB0F1C
:10710000661F771F881FD2F790480C941838092EF5
:107110000394000C11F4882352F0BB0F40F4BF2BF2
:1071200011F460FF04C06F5F7F4F8F4F9F4F089532
:10713000EF93E0FF07C0A2EA2AED3FE049EC5FEBE6
:107140000E94ED350E9487380F90039401FC9058FF
:10715000EBE3F1E00C94223A57FD9058440F551F91
:1071600059F05F3F71F04795880F97FB991F61F0C9
:107170009F3F79F087950895121613061406551F40
:10718000F2CF4695F1DF08C0161617061806991FAC
:10719000F1CF869571056105089408950E94B43871
:1071A000A0F0BEE7B91788F4BB279F3860F4161625
:1071B000B11D672F782F8827985FF7CF8695779531
:1071C0006795B11D93959639C8F30895E894BB2748
:1071D00066277727CB0197F908950E94D13708F4E5
:1071E0008FEF08959B01AC0160E070E080E89FE3C1
:1071F0000C94D5360E94B43858F19E5760F19851DE
:10720000A0F0E9F0983020F5092E9927660F771F36
:10721000881F991F0A94D1F712C0062E672F782F66
:107220008827985F11F4000C07C0993FB4F3869546
:10723000779567959395D9F7611D711D811D3EF472
:1072400090958095709561957F4F8F4F9F4F0895D2
:1072500068940C94E7380C94E6380E9440390C94FA
:1072600087380E944E3838F00E94553820F0952318
:1072700011F00C94F5370C94243811240C94E73851
:107280000E94AC3870F3959FC1F3950F50E0551FE5
:10729000629FF001729FBB27F00DB11D639FAA276B
:1072A000F00DB11DAA1F649F6627B00DA11D661FBA
:1072B000829F2227B00DA11D621F739FB00DA11DDB
:1072C000621F839FA00D611D221F749F3327A00D95
:1072D000611D231F849F600D211D822F762F6A2F31
:1072E00011249F5750409AF0F1F088234AF0EE0F96
:1072F000FF1FBB1F661F771F881F91505040A9F7C3
:107300009E3F510580F00C94F5370C94E7385F3FB1
:10731000E4F3983ED4F3869577956795B795F795FE
:10732000E7959F5FC1F7FE2B880F911D9695879576
:1073300097F908950E94B438E8F09E37E8F096393E
:10734000B8F49E3848F4672F782F8827985FF9CFD4
:1073500086957795679593959539D0F3B62FB1704B
:107360006B0F711D811D20F4879577956795939517
:107370000C94FB370C9416380C94E7389F930E94BA
:107380005E380F9007FCEE5F0C94983819F416F4F1
:107390000C9424380C9416380E94B438B8F399230E
:1073A000C9F3B6F39F57550B87FF0E941B3A002481
:1073B000A0E640EA900180585695979528F4805CA5
:1073C000660F771F881F20F026173707480730F40D
:1073D000621B730B840B202931294A2BA695179425
:1073E0000794202531254A2758F7660F771F881FF5
:1073F00020F026173707480730F4620B730B840B15
:10740000200D311D411DA09581F7B901842F9158A0
:10741000880F9695879508959B01AC010C942D39A2
:107420000E94CE3830F09F3710F40C94E7380C945B
:10743000FB370C94163891505040660F771F881F09
:10744000D2F708959F938F937F936F93FF93EF935A
:107450009B01AC010E942D39EF91FF910E942738CA
:107460002F913F914F915F910C942D39991B79E0A9
:1074700004C0991F961708F0961B881F7A95C9F7C4
:1074800080950895AA1BBB1B51E107C0AA1FBB1F13
:10749000A617B70710F0A61BB70B881F991F5A95A0
:1074A000A9F780959095BC01CD010895A1E21A2E0F
:1074B000AA1BBB1BFD010DC0AA1FBB1FEE1FFF1F98
:1074C000A217B307E407F50720F0A21BB30BE40BE8
:1074D000F50B661F771F881F991F1A9469F760952F
:1074E0007095809590959B01AC01BD01CF010895E9
:1074F000EE0FFF1F0590F491E02D09940E94893A48
:10750000A59F900DB49F900DA49F800D911D1124F7
:107510000895A29FB001B39FC001A39F700D811D6C
:107520001124911DB29F700D811D1124911D08958C
:10753000FB01DC0104C08D910190801921F44150C0
:0E7540005040C8F7881B990B0895F894FFCFB0
:00000001FF
